:020000040800F2
:1030000000800020CBB7000845B5000847B5000890
:1030100000000000000000000000000000000000B0
:1030200000000000000000000000000049B500089A
:1030300000000000000000004BB50008A188000857
:10304000E9B30008EBB30008EDB30008EFB30008E4
:10305000F1B30008F3B30008F5B30008F7B30008B4
:10306000F9B30008B1880008FBB30008FDB30008FD
:10307000A1890008FFB3000801B4000803B40008E8
:1030800005B4000807B4000809B400080BB4000830
:103090000DB400080FB4000811B4000813B4000800
:1030A00015B4000817B4000819B4000823B80008C4
:1030B0001BB400082BB800081DB400081FB400089A
:1030C00001000000000000000A00000000000000F5
:1030D0006400000000000000E803000000000000A1
:1030E0001027000000000000A08601000000000082
:1030F00040420F0000000000809698000000000091
:1031000000E1F5050000000000CA9A3B0000000045
:1031100000E40B540200000000E8764817000000AD
:103120000010A5D4E800000000A0724E18090000AD
:1031300000407A10F35A00000080C6A47E8D030080
:103140000000C16FF286230000008A5D78456301AC
:10315000000064A7B3B6E00D0000E8890423C78A25
:10316000034C206804348047FBE701F0BFFFFEE713
:04317000B4C50008DA
:10317400014802490160704708ED00E00030000892
:10318400B0B51E4D2C1F20688006400F411E032938
:1031940022D81B487944097949008F442301171A1E
:1031A400296803220A40032A00D0164829684906E0
:1031B400490F491C06F020FF29684904490E484379
:1031C4002968490F491C06F017FF0BE07D20000217
:1031D40008E00120C00305E00C3D28688004410F8D
:1031E4000848C84008490860226892093C231340F3
:1031F400064AD258D0400860B0BDC0460C10024008
:1032040000127A000024F4005C0B002034B20008A1
:1032140010B5816A8B6D8A6D5024234205D0D20685
:1032240002D4096D496B884710BD012043021A433B
:103234008A650A68D3681B059B0F02D0104908678A
:1032440010BD8B7E002BF9D113681B07F6D593684C
:103254005B0709D4583153680C24A3435360FF23FC
:1032640002330A689A4305E08A6D202313438B6571
:10327400CA6D5C3102430A600149086710BDC0464B
:04328400E809002035
:10328800F0B587B005460020049006900124E602B8
:10329800E94A1068E949884206D03246AC32E84823
:1032A800E84907F001F8E44A2868E74988420DDC54
:1032B800F449884218DDF44988422ADCF6498842F4
:1032C80042D0F64988423FD0F5493BE0DF49884281
:1032D80014DDDF49884224DCE149884234D0E149E1
:1032E800884231D0E0492DE0EE49884221DDEE499F
:1032F800884229D0012827D0EC4923E0DB498842BD
:103308001CDDDB4988421FD0DA4988421CD0DA49E3
:1033180018E0DE49884217D0DD49884214D0DD49DB
:1033280010E0CC4988420FD0CB4988420CD0CB4919
:1033380008E0DF49884207D0DE4903E0CF498842E8
:1033480002D0CF49884269D10595A868002809D0DC
:10335800D949884206D03246AE32B948B94906F052
:10336800A3FFB54A3546106904263043D34FB84207
:1033780007D105984068401E02281AD32A46B3325E
:1033880012E0D069401E082806D32A46B732AC4856
:10339800AC4906F089FFA84A059840680221C8414F
:1033A800082806D32A46B932A548A64906F07CFF64
:1033B800A14A5423D05C012802D1022007B0F0BDF5
:1033C800D45410688168490717D41169059A52685E
:1033D800022A17D104221143B9422BD1B849C94353
:1033E800059A1268D3430B43816A194054238162BA
:1033F8000024002A23D4904AAAE0906D202101439A
:103408009165A5E003933143B942AD4F24D1059CA2
:1034180021680F40826A3A4382628BE03246AD32BD
:103428008748884906F040FF834A0595A868002820
:103438008ED197E7059802680024002ADBD5A248B8
:103448000168994B9A424FD09A4B9A424FD0984B69
:103458009A4255D1052248E01F2313400F240194B6
:103468009C407549096EA143029105990968394242
:1034780037D0CF07049F4BD18F0744D44F0744D48C
:103488000F0744D4CF06374642D48E0600D5BAE09B
:103498004E0600D5B9E00E0600D5B8E0CE0500D539
:1034A800B7E08E0500D5B6E04E0500D5B5E0294257
:1034B80000D0B4E0CE0400D5B3E08E0400D5B2E06D
:1034C8004E0400D5B1E00E04019F21D4CE0300D5EF
:1034D800ADE08E0300D5ACE04E03F6171227374057
:1034E80016E04E00F70E13E00322920501E00322D6
:1034F800D2051140072292050368934359180160C9
:103508004D4A542324E0012702E0022700E0032764
:103518009F40029D2F43484E37669208F6699642AF
:1035280007D9E243846A14408A00120F9A40224362
:103538008262059C0A0243699343A4681440614A65
:1035480022401A4342610024002906D43A4A039BC8
:103558000498D054204607B0F0BD01265A480068A8
:103568000722930502461A40514FB94230D1F70558
:1035780005463D402CD154490868984302433A43D4
:103588000A6052480068524906F034FD0C21414354
:10359800481C069006980028D8D0274A039B06980E
:1035A800401E069006980028D2D00698401E069025
:1035B80006980028CCD00698401E06900698002849
:1035C800C6D00698401E069006980028E7D1BFE7A7
:1035D800354DA9420AD1370605463D4006D13A493C
:1035E8000868984302433A430A60AFE7314DA9425D
:1035F800ACD1B1050840A9D1334D2868984302439E
:103608000A432A60A2E7052782E7062780E70727FB
:103618007EE708277CE709277AE70A2778E70B2758
:1036280076E70C2774E70D2772E70E2770E7102757
:103638006EE711276CE7C046640A002000240140A9
:10364800F2C0000868BE0008FF000020FF1F003419
:10365800FFFF004000000140000002440000044851
:1036680000200034004000380080003CFF030028A0
:10367800000400280008002C001000300001002081
:1036880000020024030000081F000014200000149A
:10369800400000188000001C040000080800000C0E
:1036A80010000010FF3F00B8004000B802000004FE
:1036B800001000B0002000B404FFFF0704000080E1
:1036C800FFFF070000FFFF07082701405C0B0020F1
:0436D800400D03009E
:1036DC00F0B58DB00446002306930120002C00D1D8
:1036EC00D2E121680A68002A00D5CDE103930427B2
:1036FC003943FF250235404EB14203D120690028E1
:10370C0008D113E03D483E492A4606F0CBFD20691E
:10371C0000280BD001210A02904207D049028842AE
:10372C0004D06A1C3548364906F0BCFD6069F84186
:10373C00092804D3AA1CD648D64906F0B3FD0127A4
:10374C00F803E1690143814204D0EA1CD048D14915
:10375C0006F0A8FDB904E06808430191884204D042
:10376C002A1DCB48CB4906F09DFDA0691021C8410C
:10377C00042804D36A1DC648C64906F093FD206A86
:10378C00C549884208DC002814D03905884211D07C
:10379C00790588420ED008E0B90588420AD0F905AF
:1037AC00884207D03906884204D0AA1DB848B949C6
:1037BC0006F078FD606A322800D96DE07844007913
:1037CC00400087441F696969696969696969696940
:1037DC0069696969691F1F696969696969696969E1
:1037EC0069696969691F1F696969696969696969D1
:1037FC0069696969691F1F0004020140F2C0000871
:10380C00EEBA0008606800280DD0F90288420AD090
:10381C000321C902884206D02A4608329C489D4999
:10382C0006F040FD606822462832002812D0A068BD
:10383C0002280FD3B90388420CD005210903884212
:10384C0008D00B359248934916462A4606F02AFDB5
:10385C0032468E4E0492507800284FD10025E562F6
:10386C0015700C950B950A95099508950520000780
:10387C002168B14219D0894A91423FD188490A68DE
:10388C003A430A6009683940079102210891079967
:10389C00F902059102901EE0EA1D7D487D4906F073
:1038AC0001FD60680028B0D1BDE77D490A683A4344
:1038BC000A600A683A400792079A0A6802231A4378
:1038CC000A600968194007910C21089107997549FC
:1038DC000291202105910A950321099108AE3146E8
:1038EC0000F0E6FA07200C900B950A95022009903F
:1038FC00059808900298314600F0DAFA0597256889
:10390C00286802902A686849114026460C364CCE2D
:10391C001E43A369E769206A3043184338431043B8
:10392C000843286061680320C00281425B4E09D0C5
:10393C000598C20291420DD1306890433060716895
:10394C0011430DE00598C002316801433160716884
:10395C00814305E03068554A104030607168114071
:10396C00039F7160A16801290DD0052000038142DD
:10397C000ED005988203914212D13068104330600A
:10398C007168914312E0059880033168014303E0AC
:10399C00059880033168814331607168014305E00B
:1039AC003068434A1040306071681140716028687B
:1039BC008006800F26D030200299014022D13D484C
:1039CC0000683D4906F014FB14214143069106980A
:1039DC00002817D00698401E06900698002811D093
:1039EC000698401E0690069800280BD00698401E9C
:1039FC0006900698002805D00698401E069006985A
:103A0C000028E7D1B5420FD0019D616A8A072B4887
:103A1C0010D0CB062A4B11D41C68AC431C608C060E
:103A2C0011D55C682C4310E005984504616A8A073F
:103A3C002248EED10168A943016019E01C682C43AF
:103A4C001C608C06EDD45C68AC435C60DD601D6171
:103A5C00002A08D40268AA430260C90708D0011FD3
:103A6C000968294307E002682A430260C907F6D1B6
:103A7C00011F0968A943049A001F016050780028AF
:103A8C0001D10598507038460DB0F0BD04020140CC
:103A9C00F2C00008EEBA0008FFFF3F000002014030
:103AAC0034100240000400500F7400FEFFF7FFFFBB
:103ABC00FFBFFFFF5C0B0020400D03008418024089
:043ACC00001802409C
:103AD00070B582B00026019600280DD0054600681A
:103AE0000168002908D4042108432149884206D1ED
:103AF0002920285C01280BD0012002B070BD1D4890
:103B00001D491E4A06F0D4FB2920285C0128F3D168
:103B100028682935016801220A43026002202870C2
:103B200017480068174906F069FAC000019001982B
:103B300000281AD00198401E01900198002811D049
:103B40000198401E0190019800280BD00198401E5A
:103B500001900198002805D00198401E019001981D
:103B60000028E7D1304602B070BD02B070BDC0463B
:103B700004020140F2C00008EEBA00081F03000072
:083B80005C0B0020400D030066
:103B8800F0B585B0574C2178002902D0022005B045
:103B9800F0BD02900393012727707D20C100606A61
:103BA800049141183E04504D2868304216D0636A8B
:103BB80003208B421AD22B6833420FD0636A8B42A0
:103BC80014D22B68334209D0636A8B420ED22B6819
:103BD800334203D0636A8B42E6D307E0286843493F
:103BE8004B1C01932B600842384603D000212170FA
:103BF80005B0F0BD606A049941180120009087045F
:103C08002868384216D0636A03208B42EED22B68AC
:103C18003B420FD0636A8B42E8D22B683B4209D003
:103C2800636A8B42E2D22B683B4203D0636A8B42C1
:103C3800E6D3DBE7686800990843686002990A6080
:103C4800BFF36F8F03984860606A04994118286829
:103C5800304216D0626A03208A4219D22A68324258
:103C68000FD0626A8A4213D22A68324209D0626A45
:103C78008A420DD22A68324203D0626A8A42E6D367
:103C880006E028680199296018490842009807D079
:103C98006968009A914369600021217005B0F0BD00
:103CA800606A049941182A6800203A42F0D0636A91
:103CB80003228B4213D22B683B42E9D0636A8B42C2
:103CC8000DD22B683B42E3D0636A8B4207D22B6844
:103CD8003B42DDD0606A88421046E4D3D8E703202F
:103CE800D6E7C046E809002010200240FAC30000C9
:103CF800F0B587B00446684D287C002804D1674891
:103D08006749A02206F0D0FA2878002802D00220BD
:103D180007B0F0BD0594012129707D20C200686AB2
:103D2800069282180C045F4E3068204219D06B6AE4
:103D38000320934211D23368234212D06B6A934214
:103D48000BD2336823420CD06B6A934205D2336896
:103D5800234206D06B6A9342E6D30021297007B04C
:103D6800F0BD3068504B5A1C049232601842084625
:103D7800F3D1686A069941180120039087043068D6
:103D8800384216D06A6A03208A42E6D232683A423A
:103D98000FD06A6A8A42E0D232683A4209D06A6A27
:103DA8008A42DAD232683A4203D06A6A8A42E6D351
:103DB800D3E70022D04305990860287DA96C08182C
:103DC80081425AD201924029029106D3334834499C
:103DD800364A06F069FA0299334B7068344A104043
:103DE800C9000143A01C08437060686A069941181D
:103DF8003068204216D06A6A03208A4240D232686C
:103E080022420FD06A6A8A423AD23268224209D0E4
:103E18006A6A8A4234D23268224203D06A6A8A4283
:103E2800E6D32DE0306804993160184227D1686ADA
:103E3800069941183068384216D06A6A03208A42C7
:103E48001ED232683A420FD06A6A8A4218D2326861
:103E58003A4209D06A6A8A4212D232683A4203D098
:103E68006A6A8A42E6D30BE0287DA96C0818029991
:103E7800491C8142A7D3019805E0002003E003987C
:103E88000599029A0A6071680222914371600021C3
:103E9800297007B0F0BDC046E8090020F2C000084C
:103EA80058BB000810200240FAC30000520200006C
:043EB80005FEFEFF06
:103EBC00F0B58DB00B4604460B20000721180A20E4
:103ECC00C141039104290C9307D3052905D09848C7
:103EDC009849B12206F0E6F90C9B1868010C02D146
:103EEC0080B2002805D192489249B22206F0DAF944
:103EFC000C9B58689049884207941CDC122800D906
:103F0C000BE1012181408D48014200D105E1986807
:103F1C00032805D386488749B42206F0C3F90C9BC5
:103F2C001A68002A00D1EAE0012005908B488442EF
:103F3C000FD005200EE08249884200DDE1E0844983
:103F4C008842E4D083498842E1D083498842DED05C
:103F5C00E3E003200190059D2804029000270B97B5
:103F6C003C46099711E021437160089C1A68104681
:103F7C00E840BF1C0B99091D0B9108346D1C099965
:103F8C00491C0991002800D1B9E0681E059E0A90D1
:103F9C0086403240EAD0586812280492089423D8FC
:103FAC0001218140704A11421ED0D868042806D3E2
:103FBC00C4225F485F4906F075F90C9BD868B8407D
:103FCC000321B940079CA2688A430243A260586847
:103FDC00C206D20F0A9B9A406368B34313436360D3
:103FEC000C9BCA433E4605E00321B940CA430999DC
:103FFC004E00079CE168069211409A68B2400A4351
:10400C00E2601021014312291DD10398042841D2EA
:10401C001869082806D3DD224548464906F042F9BE
:10402C000C9800691C210B9A11400F228A400A9BA4
:10403C00DB089B00E3181C6A944388402043079CD0
:10404C0018620C984068226806990A4003210346BE
:10405C000B40B340134323600C9BC000089C85D5D8
:10406C00182020400F2383400A9A8A433C4EB118F3
:10407C000A6E9A43603105231B07079C9C4212D0A1
:10408C003A4B9C4211D03A4B9C42019B049C0ED162
:10409C0002230CE00528BBD0DC222548254906F07C
:1040AC0001F90C9BB4E7002300E00123049C83403E
:1040BC0013430B602B4801680C9B5868029A104202
:1040CC0001D0214300E0A143264A116051688203CC
:1040DC0001D5214300E0A143224A51603168C2025C
:1040EC0005D5214331607168800206D53BE7A143B9
:1040FC0031607168800200D535E7A14334E70DB01B
:10410C00F0BD1049884200D101E70F49884200D127
:10411C00FDE60E49884200D1F9E605480549B3226F
:10412C0006F0C0F80C9B9868032800D3F2E6F7E67B
:10413C00F2C00008C6BB0008FFFF10100F000600FD
:10414C00FFFF21100000221000003110000032107F
:10415C00000011100000121000002110000C005083
:10416C0000180240801802400600060000040050AF
:04417C0000080050E7
:10418000F0B581B00446744B00280CD0201F0221EA
:10419000C84103280CD88000704908581946042CDF
:1041A0000BD175310AE01946743118466E3005E0BE
:1041B000184673301946042CF3D077310778186B02
:1041C0000D780126B107009188420BD064498842DE
:1041D00008D0644988420BD102212246CA41062AEE
:1041E0000FD21EE002212246CA41042A09D218E059
:1041F000002C02D15C49884213D05C49884200D12E
:10420000A4E05B494118B002814348424841002C78
:1042100001D1002805D157485749584A06F048F8B7
:104220004D4B012F00D083E0012D00D080E0002C09
:104230000FD0211F0220C14103291DD879440979DB
:1042400049008F44011E23296F215854042C21D189
:1042500026E06E2002211954742019541D6B484A1F
:10426000954223DC0098854238D03D48854235D0C0
:104270003D48854232D029E073215854042C09D19D
:104280000EE070215854042C04D109E071215854D7
:10429000042C05D0772104E072215854042CF9D164
:1042A000752158541D6B364A9542DBDD35488542F1
:1042B00006DC2C48854211D02C4885420ED005E002
:1042C000314885420AD03148854207D029482A49D9
:1042D0002F4A1F4605F0ECFF294A3B4602212046A3
:1042E000C841062826D21F2004403046A040296A33
:1042F00081432962296A01432962186B904206DCD6
:104300000099884209D01649884206D00DE0174925
:10431000884202D01349884207D182681D49114062
:10432000062905D03204914202D001683143016070
:1043300001B0F0BD0F28D6D01548421C0D480E49DB
:104340001F4605F0B5FF0E4A3B46CCE7042121434A
:10435000042900D165E754E76C090020E4B20008A5
:1043600000040040002C01400020004000400140BB
:1043700000BCFEBFF2C00008A3BF00082408000074
:10438000FF2B0140FF430140004401400048014031
:08439000F41D0000070001000C
:10439800F0B583B00E4604468548006B854D8649C6
:1043A800884209DD8549884211DC8749884219D04D
:1043B8008649884216D010E001218907884211D029
:1043C800834988420ED0834988420BD005E07C4956
:1043D800884207D07B49884204D07F487F492A46D3
:1043E80005F062FF20680A2840D8012181407C48F6
:1043F80001423BD06068401E032804D3AA1C7648BB
:10440800764905F051FFA0680227F841042804D333
:10441800EA1C7148714905F047FFE068102804D389
:104428002A1D6D486D4905F03FFF6C226049885C84
:10443800012800D1B9E001278F54042E02921FD021
:10444800002E28D1096B086AB84308625A4881428D
:104458008D69E0680190226860680B6A4FDCBE07CE
:10446800B14252D05A4EB1424FD083E06A1C5A48EA
:104478005A4905F019FF6068401E0328BED2C2E7FA
:10448800086B4D49884244DCB90788424FD05049EF
:1044980088424CD043E0086BB90788420DD04C499C
:1044A80088420AD04849884207D03A354A484B4999
:1044B8002A4605F0F9FE3E48006B3903026A8A4332
:1044C800026261680902474A0A40E168090389B241
:1044D8008918F3221202C36993430B43016AC3612B
:1044E8000522520323681B0313409143C918016234
:1044F80003218902C2698A43C2611C3037E0334E06
:10450800B14202D0304EB14234D10326B5430543FF
:1045180031E02D4988420AD02C49884207D01A3503
:104528002D482E492A4605F0BFFE2148006B016A36
:10453800102291430162616809022A4A0A40E1682F
:10454800090389B28918F3221202836993430B4342
:10455800016A836122681201A0231A4099438918CD
:1045680001620321890282698A4382611830A16845
:10457800090213E03D4308461830F026B543019E72
:104588003601F6B2AD198D610A252A40AB439A1857
:104598000A628A690C239A438A61A1680027044A3F
:1045A800029BD75402680A430260384603B0F0BD44
:1045B8006C090020EA0F0000FF2B0140FF43014077
:1045C8000044014000480140002C014000400140E7
:1045D8000004004000200040F2C00008A3BF00080B
:0845E80005040000000FFFFFB5
:1045F000F0B583B09748401C974F79688142974E39
:1046000004D397489749324605F052FEB86800280F
:104610000BD001210A03904207D00907884204D039
:10462000721C8F488F4905F043FEF86839688E4C3C
:10463000A14212D00C21C841042805D332460832C9
:104640008748884905F034FE0120C002396A0143D9
:1046500081420CD03246093205E00121490308436A
:10466000884204D0321D7E487E4905F021FE38691B
:1046700000280DD001218902884209D00321490276
:10468000884205D032460C327548764905F010FE56
:1046900078690C25002801D0A84305D032460D3298
:1046A0006F48704905F004FE0195B8690821C841BA
:1046B000042805D332460E3269486A4905F0F8FDF0
:1046C00001200290C503F8692843A8424FD1786AB7
:1046D0000C2805D31036F048F049324605F0E8FDC5
:1046E0003E683168EF480840B9683A690A437B6917
:1046F0001343F9690B437A6E1A4302433260032075
:104700000090000372688243F868104370600022D2
:10471000A642104600D0386ABB690343B068E24C39
:1047200004401C43B460F06A0F2398433C467B6A04
:104730001843F062DD4886420DDDDD488642D84FE1
:1047400026D0BE421DD0DB4886420BD1DC48C06C6F
:104750008007000F1AE0D84886425FD0D7488642CB
:10476000CF4F15D01022D848BE4214D160E0324657
:104770000F32C948C94905F09BFD786A0C28A9D2B7
:10478000AEE7CF48C06C000A019A1040CD4A1258DB
:10479000CD48BE424CD0A94220D1082A00D974E0AD
:1047A000274652007A4492885200974408006301D9
:1047B000360163017C006301630163018800C34823
:1047C0000068BF490968890A1C220A40C049895803
:1047D0001F220A40D04000D01FE14AE1082A54D8E5
:1047E000274652007A4492885200974408004301B9
:1047F000330143016A004301430143017600B3489A
:104800000068AF490968890A1C220A40B0498958E2
:104810001F220A40D04000D01CE12AE1A848C06C09
:10482000019A1040A74A12589D4FA748BE42B2D1E4
:10483000082A2AD8274652007A4492885200974480
:1048400015001901C60019012600190119011901E5
:10485000C400C04600127A00DC080020150C0000DD
:10486000F2C0000830BC0008008000409748006893
:1048700093490968890A1C220A40954989581F22D0
:104880000A40D04000D0A2E0F3E02746F2E08C4C92
:1048900021688906490F22D0226838210A40082A57
:1048A00023D17C4893E0864C21688906490F3CD08F
:1048B000226838210A40082A43D17648ADE02846CC
:1048C000ABE07F4C21688906490F34D0226838213B
:1048D0000A40082A55D16F48BCE02846BAE0083C97
:1048E00021688904490FC84071E022680A40102AF3
:1048F00067D11D466168009A11400329654A00D0BE
:10490000024660684006400F411C104605F076FBE9
:1049100061684904490E48436168490F491C05F024
:104920006DFB2B46002852D1A3E0083C2168890486
:10493000490FC84071E0083C21688904490FC8400C
:1049400088E022680A40102A5CD11D466168009AFE
:10495000114003294F4A00D0024660684006400FCC
:10496000411C104605F04AFB61684904490E484362
:104970006168490F491C05F041FB2B4600284CD1CA
:1049800077E022680A40102A59D11D466168009AD2
:10499000114003293F4A00D0024660684006400F9C
:1049A000411C104605F02AFB61684904490E484342
:1049B0006168490F491C05F021FB2B46002849D1AD
:1049C00057E02068084020285CD10120C00359002E
:1049D000404A515A05F012FB7A68009951438842C7
:1049E00048D31103884245D8010E54080002002321
:1049F0000019594105F026FB38494118384A9142BF
:104A000035D337E0206808402028284605D02068A4
:104A1000084018282CD17D20000259002D4A515AF7
:104A200005F0ECFA400079684A08101805F0E6FA3B
:104A3000294901401ED00007400F084317E02068B5
:104A400008402028284605D02068084018280FD1A3
:104A50007D20000259001F4A515A05F0CFFA7968AB
:104A60004A08101805F0CAFA80B2102802D3F06084
:104A7000002002900020386778671A48B8660298CC
:104A800003B0F0BD206808401828F1D17D20000255
:104A90009DE7C04600127A00F2C0000830BC000852
:104AA00000800040F369FFCFFFF4FF11FF4B00408F
:104AB000004C0040003801400044004000480040E5
:104AC0000810024094B200080024F4005C0B00209F
:104AD00074B2000866B90008F0FF000000FDFFFF97
:084AE00000FD0F0001000100C0
:104AE80070B5774DA86A010A764C0FD1C10715D168
:104AF800810728D441073CD4010750D4C10664D4A7
:104B0800810678D4400600D58BE0C0E06E486F4936
:104B1800224605F0C9FBA86AC107E9D001214E0465
:104B2800E96A0A463243B24206D0621D66486749BE
:104B380005F0BAFBA86AE96A2A685368B3430B43CD
:104B480053608107D6D501210E04296B0A463243EA
:104B5800B24207D022460C325B485C4905F0A4FB00
:104B6800A86A296B2A685368B3430B43536041070B
:104B7800C2D501218E04696B0A463243B24207D07E
:104B8800224613325048514905F08EFBA86A696BDA
:104B98002A685368B3430B4353600107AED501211C
:104BA800CE03A96B0A463243B24207D022461A32D4
:104BB8004548464905F078FBA86AA96B2A685368F6
:104BC800B3430B435360C1069AD501210E03E96B29
:104BD8000A463243B24207D0224621323A483B497C
:104BE80005F062FBA86AE96B2A689368B3430B4334
:104BF8009360810686D501214E03296C0A4632430B
:104C0800B24207D0224628322F48304905F04CFBE3
:104C1800A86A296C2A689368B3430B4393604006DB
:104C280035D528682A49884208D02A49884205D0BB
:104C380022462F322448254905F036FB0120060577
:104C4800696C08463043B04206D0224630321E48CE
:104C58001E4905F029FB696C28684268B2430A437B
:104C68004260B14213D1A96C15220B46D341042BE3
:104C780007D3224635321448144905F015FBA96CB0
:104C8800286803225205436893430B434360282056
:104C9800285C000612D50120C604E86C01463143A1
:104CA800B14206D03D3408480849224605F0FCFACE
:104CB800E86C29684A68B24302434A6070BDC0463E
:104CC800DC080020E10C0000F2C0000830BC00083D
:084CD8000044004000380140D7
:104CE000F0B581B08C20364900220A50354B5C6A01
:104CF00008680168090716D5C169890213D4012122
:104D00004F050091CE02304D02E0C16939420AD10F
:104D1000596A091BA94201683DD84907F5D5C169FF
:104D20003142F2D018E00168490728D5C16949022B
:104D300025D401218F050091CE02234D02E0C169E7
:104D400039421CD1596A091BA942016823D8490775
:104D5000F5D5C1693142F2D006620D2149010368DF
:104D60008B4303608168009B9943816084202021EC
:104D7000134C215020468C302346883318E0842081
:104D800020210F4C215088202150E26610468021BE
:104D9000625401B0F0BD0D235B019943016081684D
:104DA000009B99438160064C20468830234684331B
:104DB00020211960016003208021625401B0F0BD00
:0C4DC000DC080020E8090020FFFFFF01D4
:104DCC0070B58421415821291AD102465632938A52
:104DDC00002B15D00168104C02E05B1E1D040FD097
:104DEC001588002D0DD0CD692D06F6D5056D2E88B4
:104DFC0026408E62AD1C056515886D1E1580ECE78E
:104E0C0070BD0120C0058A6882438A600868402210
:0C4E1C0002430A6070BDC046FF010000A8
:104E280010B58421415821290FD1014656310A88ED
:104E3800002A0BD0026D1388094C1C4003689C6241
:104E4800921C02650888401E088010BD0068016831
:104E5800802291430160016840220A43026010BD2C
:044E6800FF01000046
:104E6C00F0B586B00168CA690F688E688823C3588C
:104E7C00222B79D105465E3520246B89002B0094BA
:104E8C0075D0224073D03246064688366B88039321
:104E9C0001231A40049205931A0217400197876D5B
:104EAC00029502E0C266A20661D5496A039A1140D6
:104EBC0039702988491E2980816D4F1C87650168CE
:104ECC00CC6962072AD0019B5D425D41E307059BDB
:104EDC0000D02B46002B04D101230B6275681D43B7
:104EEC007560049B5D425D41A307059B00D52B4675
:104EFC00002B05D102230B62736804251D437560DA
:104F0C00049B5D425D41002A059A20D4002A20D0E2
:104F1C007268002A029D01D0002272602A88002A41
:104F2C00C1D1012212020B6893430B608A68194BA2
:104F3C001A408A602022326000220267C36E012B65
:104F4C00B0D10B681025AB43029D0B60AAE72A0079
:104F5C00DED104220A627268022313437360726802
:104F6C00002A029DD8D1D9E7183108220DE02A88F1
:104F7C00002A0DD06B899A420AD2074A026705486B
:104F8C00401C8A6802408A60009A086810430860D6
:0C4F9C0006B0F0BDFEFFFFEF75B400088A
:104FA800F0B586B004460168CA690B688D68882028
:104FB800205822287BD10495019325465E35202070
:104FC80000906889002875D00098024072D0264663
:104FD800883668880390012204981040049005924E
:104FE80010021A4602400192A76D029402E0E2669E
:104FF80098065FD5486A039A104038802888401E72
:105008002880BF1CA765CB695A072AD0019844425B
:105018004441D807059800D02046002804D1012033
:1050280008627468044374600498444244419807D1
:10503800059800D52046002805D10220086270682E
:10504800042404437460049844424441002A0598A7
:1050580020D4002820D070680028029C01D00020AD
:10506800706028880028C3D1012000020A688243A2
:105078000A608868194A1040886020203060002241
:105088002267E06E0128B2D108681024A043029C70
:105098000860ACE72000DED10420086270680222B4
:1050A8000243726070680028029CD8D1D9E7183191
:1050B80008220DE0288800280DD06A8990420AD27B
:1050C800074820670548401C8A6802408A60009AA1
:1050D80008681043086006B0F0BDC046FEFFFFEF49
:0450E800DFB4000829
:1050EC0000B5C7B0AD4A1068FF21359160313791DA
:1050FC005F393291084310607D203890C400A84E6F
:10510C003068214604F074FF401E010E012700296F
:10511C0028D1A4494860A44A1368A44E3340032004
:10512C0085075B19136000238B6007230B601168E4
:10513C0031409B4E11609E490F719E4BD96839438B
:10514C00D960D96839404291429939079A680A4323
:10515C009A609A680A4042924299400296490A68BB
:10516C0002430A6003203A904202944D28461438B8
:10517C0001683092914301223B9252023492891879
:10518C00016031682868319426461836304229D09F
:10519C00062048438A4904F02BFF0221081A0328F1
:1051AC0020D0821E514251412A6832423A4600D0E8
:1051BC000A46002A16D1421E514251412A683242F7
:1051CC003A4600D00A46002A0CD1414241412A6895
:1051DC0032423A4600D00A46002A03D1001D296803
:1051EC003142DCD13397734C27462C3F3968254626
:1051FC00283D28683A9A8243382039900140102380
:10520C000846369358408018434243413B98420429
:10521C00204634380829016825D0002B23D13B9B2C
:10522C001B041943016062494B6A046814421AD189
:10523C004C6AE41A642C14D80468144213D14C6AD6
:10524C00E41A642C0DD8046814420CD14C6AE41A8C
:10525C00642C06D80468144205D14C6AE41A652CF7
:10526C00E3D372B6FEE72E964C49096807212F91BD
:10527C0009033B680B433B603B68524C23403B604B
:10528C0003681342399C01D172B6FEE73A683B9B26
:10529C001A4306232D939A433A60454A526A3B6857
:1052AC002340082B21D0424B5B6A9B1A464EB342DB
:1052BC00EAD83B682340082B17D03D4B5B6A9B1AFE
:1052CC00B342E1D83B682340082B0ED0384B5B6AC5
:1052DC009B1AB342D8D83B682340082B05D0344BDB
:1052EC005B6A9B1AB342DAD9CEE72C4A1268520792
:1052FC002CD02A4E32682F9B9A4332602C4A526A29
:10530C00264B1B685B0721D0294B5B6A9B1A2E4EE0
:10531C00B342B9D8214B1B685B0717D0244B5B6A8F
:10532C009B1AB342B0D81D4B1B685B070ED0204BA9
:10533C005B6A9B1AB342A7D8184B1B685B0705D056
:10534C001B4B5B6A9B1AB342DAD99DE73A688A43D6
:10535C003A6039688906490F3CD0386820400828E3
:10536C001A483CD039682140102900D03FE1296807
:10537C003A9A11400329389C00D0154829684906EF
:10538C00490F491C04F034FE29684904490E48436E
:10539C002968490F491C04F02BFE21E00020024033
:1053AC005C0B002010E000E020ED00E0FFFFFF00B0
:1053BC00E809002034100240000001401470004045
:1053CC0040420F00FFF0FFFF8813000000127A002C
:1053DC000024F40000688004410FCB48C840389C7E
:1053EC00396889093C252940C84A51581F2739403A
:1053FC00C840C7490860E10004F0FAFD401EC549E9
:10540C00884200D940E7C4490979C44A5060C44C69
:10541C002068C04B18403A9B9B07C01820600026A0
:10542C0096602F981060002900D12DE720972068F6
:10543C00B849084020603398B74908712B95B94C8E
:10544C00206A3A9A90432062206A23939843206200
:10545C003B9DA805216A81432162469645962068AA
:10546C0004212C9108432060206808403D903D9811
:10547C0020682021389108432060206808403D9026
:10548C003D98206828432060206828403D903D9836
:10549C0020680221084320602068259108403D9037
:1054AC003D98206808212A91084320602068084014
:1054BC003D903D989C480F2129910161449643925F
:1054CC0014469A4842909A481838289042AF394668
:1054DC00FEF7EEFC449643942C984290954839463E
:1054EC00FEF7E6FC44964394E8031C90401C429063
:1054FC0005201F90000721903946FEF7D9FC4496F1
:10550C00439428041E90223842908B4C20463946F6
:10551C00FEF7CEFC449543962A9842902046394695
:10552C00FEF7C6FC459644964395299842907E48D2
:10553C0018383946FEF7BCFC40207D49086144967A
:10554C0043951D90429028983946FEF7B1FC754959
:10555C0048682843486048682840429042983598EB
:10556C000002764A116881431160754934980860CD
:10557C00744A2B9815542C20289015546F070C2026
:10558C002290106456649664D76416632F98506307
:10559C00906356629662101D06772C98D0619576B2
:1055AC00168369052C056848199051C2166027911D
:1055BC0051602A9890603F963E963D9626960C3AFE
:1055CC003C96D068389908432028379D06D02A4647
:1055DC0036325E485E4904F065FE5A4A106900286E
:1055EC000CD50121C907884214D05A4909E0386802
:1055FC00204020283BD13B98C003F0E60AD03B99D1
:10560C004905884206D02A4637325048504904F0A2
:10561C0049FE4C4A907E022806D32A4638324B4823
:10562C004B4904F03FFE474A906A0A211B91C8413E
:10563C00042806D32A4639324448454904F032FE40
:10564C00404A506A4449884207DC4449884215DC88
:10565C00002823D0012189021DE04149884214DC35
:10566C0013218901884219D01F99090213E0386867
:10567C002040182800D181E10020B0E611218901D9
:10568C0088420BD00921C90105E015218901884206
:10569C0004D017218901884200D072E12898105C4F
:1056AC00022806D32A463B322848294904F0FAFD41
:1056BC00244A5069042808D0082806D02A463C32CF
:1056CC002248234904F0EEFD1E4A3B980103106B5F
:1056DC0008431A91884245D1107E02284CD2507E44
:1056EC00022853D2506B08285AD2906B082861D2EA
:1056FC002B98105C022868D2D06C3843B8426FD11A
:10570C001069002876D18FE00024F40034B2000830
:10571C005C0B0020FFFFFF00E809002010E000E018
:10572C0020ED00E034100240180C0050C0E00000E6
:10573C0018080050001400500004005008E400E069
:10574C0000E100E0640A002000240140F2C00008DF
:10575C0068BE000804000080BF0400003F04000085
:10576C003F0500002A463D32FB48FC4904F09AFDF7
:10577C00FB4A107E0228B2D32A463E32F648F7493D
:10578C0004F090FDF64A507E0228ABD32A463F32F5
:10579C00F148F24904F086FDF14A506B0828A4D375
:1057AC002A464032EC48ED4904F07CFDEC4A906B03
:1057BC0008289DD32A464132E748E84904F072FD97
:1057CC00E74A2B98105C022896D32A464232E248CC
:1057DC00E24904F067FDE24AD06C3843B8428FD0FE
:1057EC002A464432DC48DD4904F05CFDDC4A106991
:1057FC00002819D03899515C022907D32A4648321F
:10580C00D548D64904F04EFDD54A106927998842EF
:10581C000AD1D069401E082806D32A464C32CE48FD
:10582C00CE4904F03FFDCE4A3898105C012809D1CE
:10583C00907E012806D12A465232C748C74904F047
:10584C0031FDC74A906D002800D0D7E0249700277F
:10585C00469745971068C349884200D0CAE0C249B0
:10586C00C8682043C860C8682040419041980868C7
:10587C000125284308600868284041904198086831
:10588C00022210430860086817921040419041981A
:10589C00449703264396E020429042AC219821463F
:1058AC00FEF706FB44971596439618954295AF481C
:1058BC002146FEF7FDFAAE4E376280200521AD4A37
:1058CC00121D32607160B760F7603061329971619E
:1058DC002E99B1613899F161306A2299C841042836
:1058EC0004D39D48A449A82204F0DCFC70683E282F
:1058FC0004D39948A049AA2204F0D4FC2521179876
:10590C00169170549D481030356829680140296003
:10591C009B488030B0649B482818142104F068FB25
:10592C00800097494118306417917164E8B20838C7
:10593C00142104F05DFB20990840189C21468140FD
:10594C00F164B068F26802433369134372691A4315
:10595C00B3691343F2691A43336A13432A681A432F
:10596C002A602546A203904218D10020179A106095
:10597C007060854A11600346014628E0389C20027D
:10598C002EE52A463A327448744904F08BFC744A6A
:10599C002898105C022800D384E68AE67068C4B2AA
:1059AC00179A1460784A1160401E032838463B460B
:1059BC0039460CD8611E88001018C367159B0B4024
:1059CC0029469940714B19607C30BC321346F76301
:1059DC00169AB5542422B75430657365B165604A84
:1059EC001665B2626A4B586835998843586028032B
:1059FC006849086054201754D765249F3B980507C5
:105A0C001468A068C00026D4A068634901402943EB
:105A1C00A16062480068624904F0EAFA40003C90D8
:105A2C003C98002817D03C98401E3C903C9800288D
:105A3C0011D03C98401E3C903C9800280BD03C98D0
:105A4C00401E3C903C98002805D03C98401E3C9051
:105A5C003C980028E7D1A0682840369B07D1404DE0
:105A6C00A96D1943A965E96D01220A43EA65A1688C
:105A7C002C9A11403A4DAA6D1A405118AA6D68D152
:105A8C0024972999C9432091F33918910A40921C03
:105A9C00AA65A268D2072E4630D1E26818239A4331
:105AAC00B3681343E3602B99725C521E534253410B
:105ABC00726823991140356C0D43776C2F43B56C8C
:105ACC003D43F16C294319432369364D1D400D4369
:105ADC0025610123DD07AA4226910ED00325AD07CF
:105AEC00AA420AD09B079A4207D0299B9B041A40D2
:105AFC002D4D2F689F43BA182A60194E326B531ED6
:105B0C009A411203337E9B03757EEF031F43B57ED0
:105B1C006B033B43F7681F4317433369002B23493F
:105B2C0002DA17311940279127990F430C49289A0B
:105B3C008A5C52003A43389E8F5D012F3AD1002D7A
:105B4C0036D007498D6D35438D65CD6D2F43CF65AF
:105B5C0030E01A43AA659BE0F2C0000868BE00085A
:105B6C00640A00200024014034100240000400505C
:105B7C00C80A0020040002403ABF0008FF7FFFFF64
:105B8C0000080240F8FFFDBF8408024044090240AF
:105B9C0008E400E000E100E0E8FFFF6F5C0B002090
:105BAC00400D030002FCFF1F08270140E8FFFF7FA8
:105BBC001E9D2A43F34E756A002D05D0379F613721
:105BCC003D401543B26A2A43E568EF4F2F40174317
:105BDC00E7602569ED4F2F4026990F4327616569D2
:105BEC002F9FBD43776B2F436761656970212891A7
:105BFC008D43B76B3F012F436761002B13D03B994B
:105C0C004D05AB421ED1DF4B1B6E1D46299E354008
:105C1C000F2DA56A0CD0F0271F40F02F08D120992A
:105C2C000D43A5620EE0A36A20990B43A36209E021
:105C3C00D44DED69AD001C351C272F402099B9407F
:105C4C001943A162E168D24B0B40934215D1002756
:105C5C00CC4BDF65996D3B9A1143259A914399651D
:105C6C00002815D03F973E97CA483D903DA8FDF7B8
:105C7C0005FB00280ED072B6FEE7C24A906D36992D
:105C8C000843259988439065D06D3B990843D065AE
:105C9C0072B6FEE72C983E90BF483D903DA8FDF7AC
:105CAC00EDFA002801D072B6FEE72A983E90BB4868
:105CBC003D903DA8FDF7E2FA002801D072B6FEE750
:105CCC0022983E90B6483D903DA8FDF7D7FA0028A3
:105CDC0001D072B6FEE7B349B34D8F65CF653A98E4
:105CEC0004048D63CF630F643E464F64349888641C
:105CFC001D98C8640C651C98486508463830279078
:105D0C00FDF7E6FC002801D072B6FEE7A749802219
:105D1C000E624E62281D41C10E604E603498886040
:105D2C00269208390846143054C00846FDF7D0FCBA
:105D3C00002801D072B6FEE79D489A49C860087CDD
:105D4C0000281DD19749487446904590994B996805
:105D5C00249A11439960996811403D913D991968B5
:105D6C00012211431960196811403D9144900320A0
:105D7C004390369842903D9842A92198FEF798F8A6
:105D8C00259888490874CE613B980874487C012892
:105D9C0001D172B6FEE72598824B1874D868C16B96
:105DAC003B9C21432D9A9143C1630168824A114067
:105DBC0001608249FE3902680A4002600168C02213
:105DCC00914301605E741C741E98401E7C4A774996
:105DDC000A634E638E63C8630E644E648E64409691
:105DEC003F963E963D962698802805D0379A3E3AA7
:105DFC007448754904F056FA6D216C480F46405CA6
:105E0C00002822D16C21694A5054116B6C4A914282
:105E1C001BD10121CA02674CE3681343E360E368BA
:105E2C0013404293429A22680A43226022680A4035
:105E3C004192022146914590449043913298429070
:105E4C00419842A92198FEF733F825985749C8552F
:105E5C00086B02683B9989072091884205D0584904
:105E6C00884202D05949884205D128998A434F4922
:105E7C00896B114300E01146554A904209DD554AA1
:105E8C00904211DC4E4A904214D0534A904211D0A9
:105E9C0070E00122920790420CD04C4A904209D0FB
:105EAC004E4A904206D065E04D4A904202D04D4A8F
:105EBC0090425FD14C4A11403C4A126C0A432699DD
:105ECC008A433A4B996C11430160D96BC162596B8F
:105EDC008162464941181B9AD141072907D83B9A40
:105EEC008A40E1210A4202D03049496C01633B9A55
:105EFC00426178232D491793CA546E231693CA54C2
:105F0C000B466E335A709A70DA701A711D465A71BC
:105F1C0074231493CA540B4674335A709A701593A5
:105F2C00DA70CA556C222392895C012901D172B6B0
:105F3C00FEE725991D4AD1553B99239BD154816885
:105F4C002B4A0A4082602B4CA0420ADD2A49884227
:105F5C0012DD214988425AD02249884257D0204923
:105F6C0052E0264988424BDC0121890788424ED0F9
:105F7C00164949E00A46A2E71849884247D0104919
:105F8C0042E0C046640A00201902FEFF02FCFFDF5B
:105F9C00E7FF3F8320000014400000188000001C25
:105FAC000001002000000020000201406C090020CC
:105FBC000074004034100240FFBFFFFFFFF0FFFFF2
:105FCC00002C0140F2C00008A3BF000800040040F0
:105FDC00FF2B0140FF4301400040014000200040E6
:105FEC000048014000440140FFFCFFFF00D4FEBF0D
:105FFC008800CEFFFF1F0040FF3F0140FF0F004015
:10600C00F649884203D0F649884200D084E1F5492C
:10601C00239A8E543B9ACA55A0420ADDF249884213
:10602C0010DDF249884219D0F149884216D0F14965
:10603C0011E0F14988420ADC0121890788420DD020
:10604C00EE4908E0EE49884208D0EE4903E0E34906
:10605C00884203D0E249884200D065E1E148806B78
:10606C002C99C841062800D9CBE03B998140572098
:10607C00014200D1C5E0DB48006C00280DD03B99F3
:10608C000902884209D03499884206D03B98C20252
:10609C00623ADD48DD4904F005F9D248806C269956
:1060AC000843802806D03B98C202613AD648D749AB
:1060BC0004F0F8F8CB48C05D002802D1C949239AF6
:1060CC0088542598C749C855086B2099884202689E
:1060DC0005D0CC49884202D0C849884205D12899BC
:1060EC008A43C049896B114300E01146C84A90426B
:1060FC0009DDC84A904211DCC24A904215D0BB4A15
:10610C00904212D006E10122920790420DD0BB4A78
:10611C0090420AD0BA4A904207D0FBE0B54A90426E
:10612C0003D0B34A904200D0F4E0BB4A1140AD4AD0
:10613C00126C0A4326998A43AA4B996C114301604D
:10614C00D96BC162596B8162B44941181B9AD14118
:10615C00072907D83B9A8A40E1210A4202D0A1497B
:10616C00496C01633B9A42619E49179BCA54169B2A
:10617C00CA546A70AA70EA702A716A71149BCA5464
:10618C00159B5A709A70DA70CA55A149884205DC81
:10619C000121890788420DD0984903E0994988422A
:1061AC0008D09249884205D09D4AA5329648974915
:1061BC0004F078F88B482399405C012801D172B621
:1061CC00FEE725988749C8553B98239A8854086B55
:1061DC008168944A0A40543282608D49884207DDB6
:1061EC008C4988421ADC8749884222D07F4919E0C1
:1061FC000121890788421CD08049884219D08049E6
:10620C0010E00120C202633A7F48804904F04AF84A
:10621C007448006C002800D031E73EE7744988428E
:10622C0007D07449884204D0774878497E4A04F0F4
:10623C0039F86C4B23981E54186B016A026A3B9D0B
:10624C00AA4302628269F0242C94A2438261259AAB
:10625C0011432A9A91430162C1681D9A9143C1600E
:10626C00C168724A1140C160DD557149884208DC31
:10627C000121890788420DD0604988420AD05749CC
:10628C0006E05749884205D05E49884202D05749FA
:10629C00884259D125985349C855239A8D54086B77
:1062AC0042685849884201D162490A4028998A4378
:1062BC0081684260564A904205DC01229207904266
:1062CC0007D04E4A03E0494A904202D04D4A9042D0
:1062DC0002D180229143816042483146239A8654F0
:1062EC00C55540963F963E9525983D903DA8FEF7A6
:1062FC004DF8002801D072B6FEE73A48006B4449CD
:10630C00884218DD434988422BDC3E49884234D010
:10631C0036492AE00A460DE73B483C49404A03F01F
:10632C00C1FF3048006B72E6D202643A36483749F6
:10633C0003F0B8FF92E60121890788421DD02F494E
:10634C0088421AD02E4910E0EA02923A2E483A4975
:10635C0003F0A8FF23482399405C01289AD172B618
:10636C00FEE72349884208D02249884205D0334AA7
:10637C00C83A2548304903F095FF1A482399405CE8
:10638C00012801D172B6FEE716484654006B816EA7
:10639C0029430E222892914381663D963DA8042103
:1063AC001191FDF7F3FF002801D072B6FEE70D48FE
:1063BC00006B1749884207DD1649884240DC1149B9
:1063CC00884249D009493FE001218907884243D0DE
:1063DC000A49884240D00A4936E0C04600100040C5
:1063EC00001400406C090020FF3F014000400140B8
:1063FC000044014000480140FF0F004000040040F1
:10640C0000200040002C0140F2C00008A3BF00088F
:10641C00FF2B0140FF430140FFFCFFFF00D4FEBFF8
:10642C00D914000088FFCEFF6C1C0000FFBFFFFFDB
:10643C00FF1300408FFF0FFF4CC30008C40900007E
:10644C00EC49884208D0EC49884205D0EB4AC83A5E
:10645C00EB48EC4903F026FFEB482399405C0128FC
:10646C0001D172B6FEE7E8484654006B816EE74AEC
:10647C001140329A11438166E549E64A0E624E623A
:10648C008E624B20179000020A6048601A98886050
:10649C00CE602E980861229848618E61CE6184206E
:1064AC0009900858002836D180200025D8490D5471
:1064BC00086890422FD10124A003D74AD168014328
:1064CC00D160D1680140429142981068204310601D
:1064DC00106820403D90469445954495022743977B
:1064EC000920400242903D9842A923912198FDF742
:1064FC00DFFC46944595449443972E9842902198FE
:10650C002399FDF7D5FCC54A1069C54908401061AF
:10651C00E006C44908602422BD48099906924250FD
:10652C00006801683B9A91430160FEF75BF8012813
:10653C001BD0B748806A002801D0FEF7CFFA3B9BEE
:10654C009903B348006882680A43826081681C9A88
:10655C00914381600168B44A0A40026001681943A2
:10656C000160FEF7B7FB002801D072B6FEE7A84821
:10657C000068AE4988420BD0AD49884208D0A54985
:10658C00884205D0349A62329D48AA4903F08AFEAB
:10659C0026989F49085C012801D172B6FEE79C4AF7
:1065AC00099806991150146820682E9020683B9B1E
:1065BC00984320602498401EA1680140A160506E51
:1065CC0023900028184612D0A568A068400F9A4F57
:1065DC00395C9A4A105CC00003F00AFD3B9028011C
:1065EC00400F395C954A105CC00003F001FD682730
:1065FC008749C8536A223B982092885226980E5499
:10660C002E9820603898099A88508848844216D071
:10661C008748844213D07F48844210D0349A9332F6
:10662C007748844903F03EFE26987949085C012896
:10663C0001D172B6FEE77648416E23910468744826
:10664C000999069A425020683B9020680125A8437E
:10665C0020602F984006A1688143A16023980028F0
:10666C00284615D0A0682E90A068400F7249095C8E
:10667C00724A105CC00003F0BBFC05462E9800016A
:10668C00400F6D49095C6D4A105CC00003F0B0FC12
:10669C005F49C85320980D5226980E543B982060A1
:1066AC003898099A88506148844214D060488442D2
:1066BC0011D0584884420ED0349A343250485D4937
:1066CC0003F0F0FD26985249085C012801D172B6FE
:1066DC00FEE74F4804684E4A099B0698D050206844
:1066EC0021680125A94321600C9569078843206026
:1066FC003898D0502698165456665148406A5049DE
:10670C00496A091A64290ED84D49496A091A64293B
:10671C0009D84B49496A091A642904D84849496A75
:10672C00091A6529EBD3E6204649474D15900D52C1
:10673C00E022464814928850A81CE42213928852F6
:10674C003A9888810C9888606720088040480478C3
:10675C00012C01D03F4800E03F4803F0A3FD0C980A
:10676C008704012C3D4C00D1C5E03D4803F09AFD57
:10677C0002F0FCF93B4803F095FD3B490E86CE85B3
:10678C008E854E858E840E84681C08853748488417
:10679C00CD8437484069002805D53648344988608F
:1067AC003548886048692648406A31994018304914
:1067BC0009691E9A114261D02149496A814265D208
:1067CC002B490969114259D01D49496A81425DD250
:1067DC0027490969114251D01949496A814255D258
:1067EC0023490969114249D01549496A8142DED3CE
:1067FC004CE0C0460044014000480140C409000080
:10680C00F2C000084CC300086C090020FFF0FFFF29
:10681C00DC080020003801403410024008E400E09D
:10682C00FFFFFF0000E100E0FFFF00FC0044004020
:10683C00008000400CC00008C0C30008B8C30008AA
:10684C00E8090020FC060020FF7F00000000FFFF8D
:10685C0048F00108B8BD000872C1000800F8010832
:10686C0079C0000868C4000800000020FFFF000089
:10687C000020024023016745AB89EFCDEB4B186933
:10688C00EB494A1C1A61084200D143E1E7484069D0
:10689C00C00704D0E54A50690C99884350613F20E9
:1068AC00E449886433980874087542A8FDF71EFA09
:1068BC00002801D0E0481CE0E048026A436A204608
:1068CC00FDF75CF9002813D1DC48826AC36A2046C4
:1068DC000830FDF753F900280AD1D848026B436BF6
:1068EC0020461030FDF74AF9002801D101F081FF54
:1068FC00D34803F0D7FCD3480069000704D4D2482E
:10690C0003F0D0FC02F032F9D04803F0CBFC02F0DB
:10691C0017FA20783899C94A5054104620306178BB
:10692C004170A1788170E178C17021790171617930
:10693C004171A1798171E179C171217A0172617A18
:10694C004172A17A8172E17AC172217B0173617B00
:10695C004173A17B8173E17BC173217C0174617CE8
:10696C004174A17C8174E17CC174217D0175617DD0
:10697C004175A17D8175E17DC1750C990D02118C5C
:10698C00B34B079559538188149A9952139A99527B
:10699C004188E22212929952C188159A995221216A
:1069AC000491CA00C18910929952832100914A0026
:1069BC00018A0F92995241218A0041890E92995273
:1069CC008121490080890D915852188B00283BD1A8
:1069DC006420319A643A97498865CA65496E0029E2
:1069EC0000D01046934A1066484248415066994A76
:1069FC00101F0B9000680104119D2840394040186D
:106A0C00684010600C981060259810600026304685
:106A1C00FDF7B0FB2846FDF7ADFB4296874CE068CE
:106A2C004290429808304290429806608A4803F09F
:106A3C0039FC607C012844D188489BE0711C844857
:106A4C00008B0E468142C3D22A9882490860844842
:106A5C001D9901607748406A7649496A091A379A44
:106A6C0091420ED27349496A091A914209D271496D
:106A7C00496A091A914204D26E49496A091A91422B
:106A8C00EAD32A987349086175481D990161002061
:106A9C00684908654865486A6649496A091A914215
:106AAC00CCD26449496A091A9142C7D26149496AF0
:106ABC00091A9142C2D25F49496A091A9142EBD331
:106ACC00BCE725985D490874C86801680C9A1143A5
:106ADC00016001683E220A40022A03D141680C9AE7
:106AEC0011434160554846740C9901745D4803F09C
:106AFC00D9FB2798FCF7E6FF002801D05A4839E06B
:106B0C005A4803F0CFFB5A48FCF7DCFF00282DD085
:106B1C0058482FE04748406A319940184349096961
:106B2C00394200D1B2E64349496A814200D3ADE60D
:106B3C003E490969394200D1A8E63E49496A814279
:106B4C0000D3A3E639490969394200D19EE6394997
:106B5C00496A814200D399E634490969394200D126
:106B6C0094E63449496A8142D8D38FE6424803F00F
:106B7C0099FB424803F096FB429641480068414914
:106B8C00884204D0404841496F2203F08BFB5420CB
:106B9C0016903B49085C012800D121E10C9816990C
:106BAC00374A5054106882688168C907339972D08B
:106BBC0025990A4033996ED181681F9A1140012999
:106BCC0029D18168324A1140259A114381603A9942
:106BDC0001601849496A8268D2075BD0154A526A2B
:106BEC00521A022A17D88268D20753D0114A526A15
:106BFC00521A022A0FD88268D2074BD00D4A526A19
:106C0C00521A022A07D88268D20743D0094A526A1C
:106C1C00521A032ADFD31A4B996D369A1143996590
:106C2C00D96D0C9A1143D965314634E000200240ED
:106C3C00FAC30000E809002098C1000800000020F9
:106C4C00FABD0008000400509ABC0008C8C3000834
:106C5C00FC060020180C00501FC1000834C10008AD
:106C6C0018080050FABC00089DB90008F8C30008C9
:106C7C006C090020B4B900080CC400080CBD000855
:106C8C00640A002000240140F2C00008E0C20008A1
:106C9C00E8FFFF7F33998268D207F34A926D40D1A7
:106CAC00189B1A40259B1A43FD4B9A65C268C36812
:106CBC003A9DAB43C360FB4B183384681C43846020
:106CCC002A40F94B8468002C2ED5429C641C4294BB
:106CDC00429C9C421AD88468002C25D5429C641C8A
:106CEC004294429C9C4211D88468002C1CD5429C36
:106CFC00641C4294429C9C4208D88468002C13D596
:106D0C00429C641C4294429C9C42DBD91698E44AF7
:106D1C001654906D36990843259988439065E3483D
:106D2C005FE13698024308E0C3681343C360DC4854
:106D3C00826D0C980243259882431698D84B1E54AA
:106D4C009A6500294CD0DA4803F0ACFAD4480068B4
:106D5C00D849884208D0309AAF32D748D74903F087
:106D6C00A1FACF4800681990199881681698CC4AF6
:106D7C00105C421E504250414907339900D40146E1
:106D8C00002900D02CE10C981699C54A505419983A
:106D9C00C068C0070FD119988068C00706D0199A2F
:106DAC009068C0490840259908439060199AD068AA
:106DBC000C990843D060429619988068C00744D15A
:106DCC00B8482F301999896801420BD0B44A906D9C
:106DDC00369908439065D06D0C990843D065FFE057
:106DEC00B248FEE0199A9068AE4908400C990843E5
:106DFC009060B3480068000221D5B2480068B249DF
:106E0C0003F0F6F8401C42904298002817D04298A4
:106E1C00401E42904298002811D04298401E429049
:106E2C00429800280BD04298401E4290429800286D
:106E3C0005D04298401E429042980028E7D19848CD
:106E4C00407E012801D001F0E3FC1698944A1654B8
:106E5C009E48401E916D0140329801439165D66564
:106E6C001C23199D2B60106D99499A4A9A4CC46247
:106E7C00026341636968369A114369600699415C03
:106E8C00012900D1A6E0014624310C9A0A704A78F7
:106E9C00012A00D09BE0259A4A70C66301680A68F3
:106EAC000C9CA2430A60826CC46C5460026D002A74
:106EBC0002D0446D856D6560199C4034056C1D4095
:106ECC000C9BAB40854D2F681F432F60119B4B6073
:106EDC008568834B102D1F4600D027468F60102DE0
:106EEC0000D01C46CC600B68289C23430B60406C84
:106EFC0003681E9C234203D00368329C2343036027
:106F0C00002A03D01068329B1843106008680C9A52
:106F1C0010430860199A9068624908401199084317
:106F2C009060704803F0BEF96F48806E3B90632808
:106F3C0001D901F04DFC6C48C06E309006E06A48F7
:106F4C0006773B98642801D301F042FC6648046F35
:106F5C00002CF4D0654BDC88DD88654A55432D0C3C
:106F6C009B277F006349CD535F48456FEF08ED1BAE
:106F7C002C193294E50855432D0CC827CD53856F39
:106F8C00EF08ED1B1F891C46ED19EF085A4A5743B1
:106F9C003F0C5A4BFF18CA23CF5221462368DF08F7
:106FAC00DB1BA788DB19DF0857433F0C1B9A5743A1
:106FBC00309ABF1ACC224F4CA7523B9A521C3B9290
:106FCC0082660667329A426785670B60B7E70E7078
:106FDC002699C163A8683349084011990843A860F1
:106FEC00474803F05FF94348818A006902F0FCF9D5
:106FFC00444945480860454808600020289048608E
:10700C001A98401E88603849496A3E4AD268002A5C
:10701C0021D0354A526A521A302A1AD8394AD268C3
:10702C00002A18D0304A526A521A302A11D8354ADE
:10703C00D268002A0FD02C4A526A521A302A08D829
:10704C00304AD268002A06D0274A526A521A302A8D
:10705C00DBD972B6FEE72B490969814206D1294872
:10706C002B49016004E0C046640A002025490861F0
:10707C001798800008900B200290400220900C98EA
:10708C00C104189181050A91C1050191C0060390B4
:10709C002048FE30059028982790239049E0C04660
:1070AC00640A0020E8FFFF7FFFF1020080C40008A3
:1070BC00C5C1000800240140F2C0000868BE0008E9
:1070CC00082701405C0B0020400D0300FFF0FFFF80
:1070DC00D3B7000821B400081532000804000240A0
:1070EC000400002050BA0008E8090020000000202D
:1070FC0088130000FC060020C4090000A8FD000055
:10710C00E6C1000800300040CCCC00005555000012
:10711C00AAAA0000D91400000020EC493B9A885020
:10712C000875EB4803F0BEF8E84800688821222275
:10713C004250E848E84901602898401CE749496AF0
:10714C00814245D3E548006D002821D0401EE3491B
:10715C0008651DD1E148406DE149012800D110318D
:10716C002A9A0A60DF49012800D110311D9A0A6061
:10717C00411E4A1E9141D94A5165127E002A31990D
:10718C0000D10021012801D0D448C16CD34801653D
:10719C00D248006E002818D0401ED049086614D181
:1071AC00CE48406ECE49012800D11031119A0A60A8
:1071BC00411E4A1E9141C94A5166012801D0CA4854
:1071CC0000E0CA480068C5490866C448406A28906F
:1071DC002798401CC149496A814201D200F073FDD5
:1071EC00BE48416A2791006F00283ED0C04DE88808
:1071FC00E988C04B5943090C9B225200BE4CA1524A
:10720C002646B64F796FCA08891A08183B90C108F0
:10721C005943090CC822A152B96FCA08891A2C46C5
:10722C002A898A18D108B54D6943090CB44BC91881
:10723C00CA23F15223682646DC081B1BB4881B1991
:10724C00DC086C43240C1B9D6C43BD6EFE6EA41BB2
:10725C00CC26A94884536C1CBC6600243C673B9824
:10726C007867BA67A248036002E0CA20A249095AAB
:10727C004820A14F385E0CB2201A0A2102F090FE71
:10728C004A21795A41433A8D8918EA221C92B95203
:10729C004C21795A41437A8D8918EC221992B952B2
:1072AC004E21795A4143BA8D8918EE22B952502297
:1072BC00BA5A4243FB8DD3182C9A3093BB525222AC
:1072CC00BA5A42433B8ED218F2231E93FA52169AA4
:1072DC00BA5A42437B8ED218F4232E93FA5256227A
:1072EC00BA5A4243BB8ED318F622BB525822BA5A12
:1072FC004243FD8E5619F822BE525A22BA5A4243C4
:10730C004620385A1018FA22B852FC22BA5A002ACF
:10731C0002D1E822784DA8523998774A105E8442FF
:10732C0003DDCE200122744D2A523A20724A105E9F
:10733C00844203DACE2000226F4D2A522B986E4ADB
:10734C00105E844203DAD02001226B4D2A523E207B
:10735C00694A105E844203DDD0200022664D2A5219
:10736C001D98654A105E844203DAD2200122624DD8
:10737C002A524220604A105E844203DDD220002251
:10738C005D4C2252C8225C483B92825A98B282428F
:10739C0006D3B0B2824203D8D420574B1B5A08E014
:1073AC00B0B2824201D9002300E00123D420524C18
:1073BC002352CE2450483294065B701E4442444102
:1073CC0088B28242339800D82046D0244A49095BBF
:1073DC004F1E7D427D410028339800D128465F1E08
:1073EC007D427D410028339806D1012D06D030987E
:1073FC0080B2824217D325E00128F8D10220384907
:10740C000861DE2001213C4A1152D420135A115B31
:10741C003298165A2C98105A30903B98125A309831
:10742C0080B282420ED2002E0CD100290AD1002B40
:10743C0008D102202A490860DE2000212E4A115270
:10744C003B98125A2C481E99405A824213D2234B15
:10745C00986B31994018596A81420CD3D621264C2D
:10746C00635A4420205A834202D2581C224B585251
:10747C001A49486A8863204D3298285A401E444263
:10748C0044414421685AD623ED5A8542339E00D09C
:10749C002646D2251848405B441E60426041002EAF
:1074AC00339C00D10446012C07D101200C4A1061F9
:1074BC00DC22114CA0523B98225A0F482E9C005BA8
:1074CC0082421FD900220C48C2521DE0C004002089
:1074DC0067BA000800300040AAAA0000E8090020A2
:1074EC00180C005018080050400A0020440A0020D4
:1074FC000000002088130000FC060020C4090000D6
:10750C00A8FD0000FC48C25A002A0FD1FA48329A52
:10751C00805A00280AD1F848405B002806D1012087
:10752C00F64A1060DC200022F34C2252FE22F24874
:10753C003092805A02282AD1F148406C012800D19F
:10754C00F4E03398EE4A10760B98006801042A9BFD
:10755C001840189C214040185840E8490860E949F7
:10756C00D164506D002800D03199E54A1165414233
:10757C0041415165E44A101F006801041D9B1840ED
:10758C000A9C21404018584010600120CCE0C01EDD
:10759C0001282AD8DA48406C022800D1C6E033987A
:1075AC00D74A10760B98006801042A9B1840189C47
:1075BC00214040185840D1490860D449D164506DDD
:1075CC00002800D03199CE4A1165414241415165A4
:1075DC00CD4A101F006801041D9B18400A9C2140D5
:1075EC0040185840106025989EE0C348329A805A43
:1075FC0001282AD1C248406C032800D196E0339868
:10760C00BF4A10760B98006801042A9B1840189CFE
:10761C00214040185840B9490860BD49D164506DAB
:10762C00002800D03199B64A11654142414151655B
:10763C00B54A101F006801041D9B18400A9C21408C
:10764C004018584010603A986EE0AB4A3B98105A7C
:10765C001C9C125B904225D9A948406C042865D02B
:10766C003398A74A10760B98006801042A9B18409F
:10767C00189C214040185840A04908603198D064AB
:10768C001065506D4142414151659F4A101F006881
:10769C0001041D9B18400A9C214040185840106062
:1076AC00119841E0944A199C125B904232D2944852
:1076BC00406C052823D03398914C20760B980068A9
:1076CC0002042A9D2840189E3240801868408B4A3C
:1076DC0010609622E264606D002800D0319A884CCC
:1076EC002265424242416265874C201F00680204B9
:1076FC001D9D28400A9E32408018684020607F48BB
:10770C000C9A0261DC20259A7B4C2252605AE05282
:10771C001F9809E02A98794908617B481D990161F5
:10772C000020774908654865754948647448007BB2
:10773C00002809D12C9870490D5A3B980E5A0020FC
:10774C00AE4205D20C9D12D2002500281ED010E0AE
:10775C006949079A885A401C88523398684F387385
:10776C006C4802F09FFD387BAE420C9DECD3002898
:10777C000CD061492E98085A3B9A895A814205D8F7
:10778C00654802F08FFD00205D4908735C49C86BA9
:10779C00624A8018496A8142339802D25848007F65
:1077AC00C043C00700D188E0339855490877486A30
:1077BC00C8635B4802F076FD4F483B99415A129AD8
:1077CC00805A814207D24C4CA152564802F06AFDB5
:1077DC003B98215A339D4848149A805A814205D9C6
:1077EC0045488152504802F05DFD339DCA26424AFD
:1077FC00915F1598105E814207DA15983E4C215224
:10780C004A4802F04FFDA15B339D3B48139A805EC2
:10781C000AB2824208DD384C139821524448114672
:10782C0002F040FDA15B339D3998334A105E323033
:10783C0009B288420EDA30480E9A805A3D4A90427C
:10784C0008D0401C2C4C0E9AA052394802F02AFD4C
:10785C00A15F339D1D98284A105E323888420ADD9C
:10786C0025480D99405A3349884204D0401C22497E
:10787C000D9A8852339D20493B98085A498D64399A
:10788C0081420ADD1C490F9A895A2A4A914204D036
:10789C00491C194A0F9BD152339D1749098D6431EC
:1078AC0081420AD214481099405A2249884204D085
:1078BC00401C1149109A8852339D1149086C1E4A7C
:1078CC008018496A814209D30D49486A08641B48EB
:1078DC0002F0E8FC002D01D001F0C4FC1848056B47
:1078EC001848854236DD184885423CDC17488542ED
:1078FC0046D017483BE0C046FC060020180C005050
:10790C00E8090020581B00001808005088130000DC
:10791C00B80B00002DBA000854BD000860EA000046
:10792C006ABD000884BD00089EBD000820C4000884
:10793C0038C40008FFFF000080EE360050C4000879
:10794C006C090020FF2B0140FF430140002C01403B
:10795C000040014001208007854211D0F648854245
:10796C000ED0F64803E0F648854209D0F54885422A
:10797C0006D0F548F549059A02F094FCF448056BDD
:10798C006C6BF448854205DC0120800785420FD0E2
:10799C00E94803E0F04885420AD0F048854207D018
:1079AC00209A1F3AE848E94902F07CFCE848056B4C
:1079BC00AE6B97204000EA4F3E52A01B17998900EE
:1079CC00785202F0B5F90446304602F0B1F901469E
:1079DC00204602F0BFF8014601F0BEFF06463B9878
:1079EC00385A02F0A5F9314602F058F802F056F96F
:1079FC000A2132902E9102F0FBFA132109017852E0
:107A0C00D8203B90385A002810D0696AD548C06AF3
:107A1C00379A953291420CD9D149309A895A00291A
:107A2C0007D1D04A1172401CD06207E0CC484018F4
:107A3C00B2E0002829D0401ECA49C862642824D369
:107A4C00C94802F02FFC0025459544950120439030
:107A5C00389F4297469542AEC44C20463146FCF7BF
:107A6C0027FAA7622F98469045954495022043909B
:107A7C00429720463146FCF71BFABA49CD6233983F
:107A8C000872086B401C086301E0B648006B0A28BA
:107A9C001CD90025B2493B980D524295B448C06898
:107AAC004290429808304290429805600420309AE7
:107ABC008852B04802F0F6FBAA490D63486B401C93
:107ACC0048633199491E88420DD80FE0A54A516B85
:107ADC00491C5163319A521E914207D9002802D099
:107AEC00401EA049086300209E4948639920450028
:107AFC009B48415B9B48007A9F4A329B934203D33D
:107B0C00002801D0012202E000299C4A1BD08918D0
:107B1C00934A515389B2652915D30026904C3B9852
:107B2C00265242969248C068429042980830429041
:107B3C0042980660022030996052914802F0B2FBE4
:107B4C0066538848007A4D218D008E49329A8A42BC
:107B5C008349495B03D8002801D0012002E00029A9
:107B6C0086481BD008187E49485380B2652815D327
:107B7C0000207B4C3B99605242907D49C9684291F0
:107B8C004299083142914299086003203099605221
:107B9C007D4802F087FB6019002101807B4840681A
:107BAC000028339904D0401E784948604142414135
:107BBC00DA256B48405B00285ED100295CD0734805
:107BCC002E994160E820664B1A5A9B2149005B5A5A
:107BDC00934229D9624C3B9EA65B6D4CA64223D2A4
:107BEC005F4C309FE75B002F1ED1721C5C4B3B9CA3
:107BFC001A53089B5B1E9BB29E4207D2584A089CA4
:107C0C003B9BD4520022574B1A63224600234293CB
:107C1C00574BDB684293429B0833429392B2429B90
:107C2C001A604F4B1A5A5B5A934223D24C483B99D9
:107C3C00405A00281ED0411E8AB20020089B9A424E
:107C4C00024600D30A4646493B9BCA52429096B222
:107C5C004A480E38864205D3319A893A3A484D49FA
:107C6C0002F020FB4248C068429042980830429093
:107C7C00429806603A48405B012813D138483B993A
:107C8C00405A4349884210D23549309A895A0029C2
:107C9C000BD142913649C9684291429908314291BF
:107CAC00429908602E483B99405A319964396422B4
:107CBC0000280B4600D013462A4CE365002800D060
:107CCC000A46284882652748406A239988420DD97C
:107CDC002449886A496A2391002807D0401E21490B
:107CEC00886203D1FC2000211D4A115226202E90BF
:107CFC001B48408B002800D1BFE127492E9A895C94
:107D0C00002900D0B9E1411E072949D84900C046D5
:107D1C007944898849008F4407004F0061004E0563
:107D2C00670081009600B0001C4802F0BBFA0020EE
:107D3C00014601F05BF99DE1000400400020004089
:107D4C000044014000480140F2C00008A3BF0008F5
:107D5C006C090020FF2B0140002C01400040014029
:107D6C00FC060020E809002049C10008000400506E
:107D7C0000000020CBB90008A1090100FFFF0000A2
:107D8C00F6B900080F2700001EBD00085C0B002090
:107D9C00DC050000D1BE0008C0040020B4BC000803
:107DAC00FA49884200D087E0F94802F07BFA0021BA
:107DBC00339801F01BF95DE1F64802F073FAF648CE
:107DCC000068F64988427DDDF549884200D187E09C
:107DDC00F449884200D183E0F34977E0F34802F09C
:107DEC0061FA00F0C3FE45E1F14802F05BFA62244F
:107DFC00F048015BF048008C814209D10020339996
:107E0C0001F0F4F86420EB49085A0853EA49088455
:107E1C00411E88415E21E74A50522BE1E74802F0AF
:107E2C0041FA6220E349085AE349098C884245D15A
:107E3C00012000020021DF4A11501018018141601D
:107E4C0001F010FA16E1DE4802F02CFA6220D94952
:107E5C00085AD949098C884230D1CA20D54A105ABF
:107E6C001599505213995052C820105A12995052C9
:107E7C001499505201F0F6F9FCE0D24802F012FAD3
:107E8C00CD48406ACC49496A0A1A3199491C8A4240
:107E9C0000D3EFE0C84A526A121A8A4200D3E9E0D2
:107EAC00C54A526A121A8A4200D3E3E0C24A526AA5
:107EBC00121A8A42E6D3DDE0C34800E0C34802F060
:107ECC00F1F9D7E0C24988420AD0C249884207D0AA
:107EDC00349A7432C048C14902F0E4F9AE480068E3
:107EEC00AD49099A069B8B50016801221C92914363
:107EFC00016000210160416019918160AA498842AA
:107F0C0000D0A7E0B649C868B64A1040C860022045
:107F1C003B90042032902A983090199D24E03B9895
:107F2C008140219F3868084338601C20329B1840E0
:107F3C00299B8340E80880003818046A9C4304623B
:107F4C00B8688843B860786890437860F86888436C
:107F5C00F8601E98851C3298083032903B98001DB2
:107F6C003B903098103030901C9EAE40314620989B
:107F7C0001403BD030980838369A1040299A8240FC
:107F8C0003202B468343984CE3181C6E144211D1EA
:107F9C006033964F3C688C433C607C688C437C60BF
:107FAC00914F3C688C433C607C688C437C601968C6
:107FBC00914319603B99891E8840219C216801439B
:107FCC0021603299091F18220A4029999140EA0828
:107FDC009200A218136A8B431362A1688143A160BB
:107FEC006168B1436160E1688143E160681C0D2800
:107FFC0029D0401E02221E90824010462099084033
:10800C00A7D01821309B1940299B8B4003212C466B
:10801C008C43754F3C19276E1F4200D07FE76034AC
:10802C00724E3768874337607768874377606E4F47
:10803C003F6887436C4E376077688743776020686A
:10804C00984320606BE7039869490860BFF34F8F32
:10805C00BFF36F8F8C205049199A0A5009980A5017
:10806C0088200A5080200A54CA6652490869898AB5
:10807C0001F0BAF900204F4948835E48007D002882
:10808C0001D1FFF756F84520C1005A483B914058A2
:10809C00042801D8FFF740F8074627255548405DCE
:1080AC00329001201E90C443B81E3090044000262C
:1080BC00514A03E0B61CB44200D1C0E04D488019CF
:1080CC00415D51408AB25208C9071DD04B494A4004
:1080DC005308D1071BD15A08D9071DD047494A402C
:1080EC005308D1071BD15A08D9071DD043494A4020
:1080FC005308D1071BD15908DA071DD03F4A51400C
:10810C004A08C9071BD11CE05308D107E3D03B49EF
:10811C004B405A08D907E1D15308D107E3D037496E
:10812C004B405A08D907E1D15308D107E3D0334962
:10813C004B405908DA07E1D14A08C90701D02F4949
:10814C004A402823C15C51404808C90758D02B49E4
:10815C0048404108C00756D14808C90758D027499C
:10816C0048404108C00756D14808C90758D0234990
:10817C0048404108C00756D14808C90758D01F4984
:10818C0048404208C00795D056E0C0463930000040
:10819C008AC00008CABC0008DC080020FF4B004065
:1081AC00004C00400080004000380140B1B3000892
:1081BC009FC00008FC060020E8090020E4BC000871
:1081CC00D8C30008B4C00008E1C000087EB900089C
:1081DC000044004000480040F2C0000830BC0008D9
:1081EC0034100240FFBFFFFF00180240801802400D
:1081FC0080E100E0C0040020FFFF000001A00000AF
:10820C004108C007A8D0FD4841404808C907A6D17D
:10821C004108C007A8D0F94841404808C907A6D171
:10822C004108C007A8D0F54841404808C907A6D165
:10823C004208C00700D13DE7F04842403AE7F80752
:10824C0042D0EF480019405D424090B24008D1073F
:10825C001DD0EA4948404108C0071BD14808C9074E
:10826C001DD0E64948404108C0071BD14808C90742
:10827C001DD0E24948404108C0071BD14808C90736
:10828C001DD0DE4948404208C0071BD11CE0410804
:10829C00C007E3D0D94841404808C907E1D141089B
:1082AC00C007E3D0D54841404808C907E1D141088F
:1082BC00C007E3D0D14841404808C907E1D1420882
:1082CC00C00701D0CD484240791C48424841CD4CB2
:1082DC003099615C3D196D1E2D782D02691892B292
:1082EC009142339900D10146012903D1C64801F0CE
:1082FC00D9FF25E0C548018B329D4A1B50425041A5
:10830C00002D339A00D00246002A19D09320450044
:10831C00BB4A3095329850558B20850000201C9517
:10832C005051D25C102A12D0062A1AD0032A25D119
:10833C00329A002A2BD0914229D08620029960E0F3
:10834C000020AF493B9A88500875FEF7EDFE329835
:10835C00002828D0814226D003270B2186261E9A7E
:10836C00AAE0329800282DD081422BD035982830A5
:10837C008621A34A115402210B20C7E0A048309952
:10838C0040181E99817026994A4042703EE06379EC
:10839C0021790902CA1811467E397C25ED43A94280
:1083AC0022D203212CE06179207900024218104678
:1083BC007C387A23DB4303279026984228D21E9AD6
:1083CC00394679E0E178A078000240189C2800D367
:1083DC0095E08D2292008A4B9A58125C022A72D038
:1083EC00002A77D18A4888E0E178A47824026118C1
:1083FC00521814469D3C9B25ED43AC4218D20221E9
:10840C0000987F4A309BD21891705070032782E0FD
:10841C00E378A078329000021993C41815192846F5
:10842C009D389B22D24390421BD202211E9A43E0DC
:10843C00734D309C2C195B00A37003236370359B28
:10844C002A33EB184C00714D2C19255C5D702518E6
:10845C006D781D70801C9B1C491C9142F5D3C71C68
:10846C0059E06000694A10184722D200644B9F58AB
:10847C008D2292009A582F3309E01E7806705E1EEA
:10848C0036784670801C9B1C641CAC4208D2165D6E
:10849C00002EF7D0022EF0D13E88002EEDD1F1E760
:1084AC00F348309A8018199AC270329A8270369AB0
:1084BC004270042200262D9FED488018309A865475
:1084CC008018417027E04722D200E94B9A58128855
:1084DC00002A11D042006079E24B98549A18237903
:1084EC005370E34A309C12191371D17000219170B2
:1084FC002D995170052109E0E04801F0D3FE359823
:10850C0028308621DA4A115402200146D84A5218E2
:10851C00309BD0544F1C39461E9881433A4602403A
:10852C00D348309BC3180C46CF4D03E09B1CA41EB4
:10853C0000D18EE0187868404508C0071DD0CB48A4
:10854C0045406E08E8071BD17508F0071DD0C748D9
:10855C0045406E08E8071BD17508F0071DD0C348CD
:10856C0045406E08E8071BD17008F5071DD0BF4DBC
:10857C0068404508C0071BD11CE06E08E807E3D033
:10858C00BA4846407508F007E1D16E08E807E3D019
:10859C00B64846407508F007E1D16E08E807E3D00D
:1085AC00B24846407008F507E1D14508C00701D034
:1085BC00AE4845405E786E407008F5072AD0AB4D4A
:1085CC0068404508C00728D16808ED072AD0A74D98
:1085DC0068404508C00728D16808ED072AD0A34D8C
:1085EC0068404508C00728D16808ED072AD09F4D80
:1085FC0068404508C00799D028E0C04601A000009B
:10860C00C0040020E7040020FFC10008FC06002085
:10861C00A4C400084508C007D6D094484540680853
:10862C00ED07D4D14508C007D6D09048454068081E
:10863C00ED07D4D14508C007D6D08C484540680812
:10864C00ED07D4D14508C00700D16FE787484540F6
:10865C006CE7002A43D0864840183099405C45406E
:10866C00A8B24008E9071DD0804948404108C0071E
:10867C001BD14808C9071DD07C4948404108C00798
:10868C001BD14808C9071DD0784948404108C0078C
:10869C001BD14808C9071DD0744948404508C0077C
:1086AC001BD11CE04108C007E3D07048414048088A
:1086BC00C907E1D14108C007E3D06C4841404808E4
:1086CC00C907E1D14108C007E3D0684841404808D8
:1086DC00C907E1D14508C00701D064484540290AC3
:1086EC00634CE019309A85548018417022982E9969
:1086FC006054BB1C1C98235098B2424242412068E3
:10870C00014680314C68202C339C00D11446002C3F
:10871C0030D10A78012A2DD00546543584686B80F7
:10872C000022CA602B80524B309D5B190365049B61
:10873C004B60436E249DAB420DD11A9B9C4203D1DE
:10874C000369002B504B00D0504B0A7043670068F4
:10875C00083001990BE01A9B9C4203D10369002B52
:10876C00474B00D0474B0A70436700682699026854
:10877C000A43026000203E4D3B9968506221394CFF
:10878C00615A334B1A8C891A4A424A41602162520F
:10879C002875DA835C20205A002801D1FEF7C9FC29
:1087AC00FC21304A1E9B5352E8215052284838492C
:1087BC008162FEF7BEFC2F4801F074FDBFF34F8FB2
:1087CC00224914392C480860BFF34F8F00BFFDE7D6
:1087DC0022480168CA08891A828889180160C90868
:1087EC001F484843000C1B9948431949C866FEF7BB
:1087FC00FAFB19481830144A516901435161506908
:10880C0014480069000701D4FEF779F8FEF77CF8EC
:10881C000F48406A199B06E00D49496A091A032959
:10882C0001D3FEF7D3FA19990968C90701D0FEF7ED
:10883C000CFB19998968C907EED19968064A114051
:10884C000C9A11439960E7E70020024020ED00E00C
:10885C00E809002000040050E8FFFF7F0000002022
:10886C00C4090000FC060020FFFF000001A000006E
:10887C00C0040020D9B300080400FA05C0C40008E5
:10888C00294E0008E7B70008CD4D000823B40008B6
:04889C00E093040061
:1088A0000248416A491C41627047C046E8090020FD
:1088B000F0B583B03848001F0568384A146820684E
:1088C00004260190304041424141106C1C2303407A
:1088D00037469F40384602952840424242410A436B
:1088E00030D0009401200226019D2A463240514298
:1088F00051419E40029A1642074600D00F46002F73
:1089000032D008210D4069426941DA40120700D592
:108910000846002826D124200021204C2154009A0A
:1089200010680E21884310600120014699401A4BBF
:108930001A680A431A60E06325216054616B0029BC
:108940000ED10FE02068800602D42068B04320607A
:1089500011490868384308601048016B002901D0AC
:108960000E48884703B0F0BD2346206880060B4AB6
:1089700006D418680A218843186025200121115463
:108980002420002111540449086830430860D16A4A
:108990000029E5D1E6E7C04604000240C80A0020ED
:1089A000F0B583B06E4D286801680291EF21CC00CC
:1089B00047686C49884204D06B486C49224601F0F4
:1089C00077FC6869042806D0082804D0621C664831
:1089D000664901F06DFC022338461840414241418E
:1089E00002981840424242410A4308D1A86DC0068D
:1089F00003D48834A86D2043A865286803600193D8
:108A0000012504203840424242410298400728464E
:108A100000D510466E0201280AD108203840434292
:108A2000434102980007284600D5184600282FD158
:108A30004B49886DC00602D4886D304388650B6849
:108A4000D8680005800F1ED14548807E00281AD1C5
:108A50001868000717D59868400709D458680C2192
:108A600088435860FF200230424C2168814307E070
:108A70003B48846D20212143816504465C34C16DEF
:108A80000120084320603A48012101670C2018604A
:108A90008023384618404442444102980006284644
:108AA00000D52046002807D1012000042C4CA16DE0
:108AB0000143A1652068036001231C02394621405F
:108AC000484248410299C905294600D50146002976
:108AD00006D15804224A916D0143916510680460E3
:108AE000394631404842484102993142294600D036
:108AF0000146002906D19804194A916D01439165F8
:108B000010680660102239461140484248410299D7
:108B1000C906294600D50146002911D1104804682C
:108B2000006B002802D0E068800708D098020C4E45
:108B3000B16D0143B165F06D01990843F0652260A4
:108B4000580307407A427A410299890401D403B05C
:108B5000F0BD1500FBD102490968086003B0F0BD03
:108B6000640A002000240140F2C0000868BE00082A
:088B7000E8090020BC0A002006
:108B7800F0B581B06A4801F097FB6A486A4D29460A
:108B88005CC85CC15CC85CC15CC85CC15CC85CC1D9
:108B9800482001262E5468206864286C401C2864EC
:108BA800624F7868002806D5384608386049016061
:108BB8006049016078687D20C1005F48426A5218A8
:108BC80033043C681C4215D0446A944218D23C686D
:108BD8001C420FD0446A944212D23C681C4209D00D
:108BE800446A94420CD23C681C4203D0446A9442C2
:108BF800E7D305E03A68514B5C1C3C601A4268D0E8
:108C08007968C90702D07968B14379603E218164E7
:108C1800067406756846FBF76BF8002800D0FEE777
:108C28000CCD474C2046083DFAF7AAFF0028FED194
:108C3800AA68EB6820460830FAF7A2FF0028FED1A0
:108C48002A696B6920461030FAF79AFF0028FED18E
:108C5800AA69EB6920461830FAF792FF0028FED17E
:108C68002A6A6B6A20462030FAF78AFF0028FED16C
:108C7800AA6AEB6A20462830FAF782FF0028FED15C
:108C88002A6B6B6B20463030FAF77AFF0028FED14A
:108C9800AA6BEB6B20463830FAF772FF0028FED13A
:108CA8002A6C6B6C20464030FAF76AFF0028FED128
:108CB800AA6CEB6C20464830FAF762FF0028FED118
:108CC8002A6D6B6D50342046FAF75AFF00281DD0E4
:108CD800FEE7426A5118B2043B68134290D0436AD7
:108CE8008B428DD23B6813428AD0436A8B4287D22B
:108CF8003B68134284D0436A8B4281D23B6813425B
:108D080000D17DE7436A8B42E6D379E7F0077968BB
:108D180001437960786800F015F801B0F0BDC046ED
:108D2800CEBD0008A4B20008680000201020024050
:108D380023016745AB89EFCDE8090020FAC300009D
:048D480000F001082E
:108D4C00F0B588B0A3490A78A34802704A784270FB
:108D5C008A788270CA78C2700A7902714A79427133
:108D6C008A798271CA79C2710A7A02724A7A42721B
:108D7C008A7A8272CA7AC2720A7B02734A7B427303
:108D8C008A7B8273CA7BC2730A7C02744A7C4274EB
:108D9C008A7C8274CA7CC2740A7D02754A7D4275D3
:108DAC008A7D8275CA7DC2750A7E02764A7E4276BB
:108DBC008A7E8276CA7EC2760A7F02774A7F4277A3
:108DCC008A7F8277C97FC17784490A782023C2546D
:108DDC004A782123C2548A782223C254CA78232386
:108DEC00C2540A792423C2544A792523C2548A795D
:108DFC002623C254CA792723C2540A7A2823C25480
:108E0C004A7A2923C2548A7A2A23C254CA7A2B2337
:108E1C00C2540A7B2C23C2544A7B2D23C2548A7B16
:108E2C002E23C254CA7B2F23C2540A7C3023C25433
:108E3C004A7C3123C2548A7C3223C254CA7C3323E9
:108E4C00C2540A7D3423C2544A7D3523C2548A7DD0
:108E5C003623C254CA7D3723C2540A7E3823C254E7
:108E6C004A7E3923C2548A7E3A23C254CA7E3B239B
:108E7C00C2540A7F3C23C2544A7F3D23C2548A7F8A
:108E8C003E23C254C97F3F228154554A1178402356
:108E9C000793C15451784123C154917842230693CE
:108EAC00C154D1784323C154117944230593C1543F
:108EBC0051794523C154917946230493C154D179F6
:108ECC004723C154117A48230393C154517A49233F
:108EDC00C154917A4A230293C154D17A4B23C15481
:108EEC00117B4C230193C154517B4D23C154917B75
:108EFC004E230093C154D17B4F23C154117C502578
:108F0C004155517C5123C154917C52240155D17C43
:108F1C005323C154117D5423C154517D5527C15540
:108F2C00977D56214754D27D5727C25507682D4A45
:108F3C00176187889782C788D782078917834789E3
:108F4C00178587895785C7899785078AD785478A63
:108F5C001786878A5786C78A9786078BD786478B4B
:108F6C001787878B5787C78B9787078CD787478C33
:108F7C00079E9753878C069E9753C78C059E9753D5
:108F8C00078D049E9753478D039E9753878D029EA2
:108F9C009753C78D019E9753078E009E9753468E0D
:108FAC005653858E1553C48ED452038F5352418F12
:108FBC005823D152818F5A23D152C18F0A4B198415
:108FCC00002902D05E2101235352C06C506008B0BE
:108FDC00F0BDC04600F001086800002020F0010838
:0C8FEC0040F00108FC060020E80900200D
:108FF800F0B583B00D460190914801F055F9914FB5
:1090080038697969904E03C6388B3080388D708006
:10901800788DB080B88DF080F88D3081388E708171
:10902800788EB081B88EF081F88E3082388F708259
:10903800788FB082B88FF082F88F30834020385A0A
:1090480070834220385AB0834420385AF08346202F
:10905800385A30844820395A71844A21795AB1845F
:109068004C21795AF1844E21795A31855021795A07
:1090780071855221795AB1855421795AF185562141
:10908800795A31865821795A71865A21795AB18686
:109098006E4C083E002D02D12146203101E03946B0
:1090A8006431098801253554F18768207064306C73
:1090B800401C30640198002804D0654801F0F4F899
:1090C8007868F064634F7868002806D53846083811
:1090D800614901606149016078687D20C000616A6A
:1090E80009182A043B68134215D0636A8B4218D2C8
:1090F8003B6813420FD0636A8B4212D23B6813421B
:1091080009D0636A8B420CD23B68134203D0636A6E
:109118008B42E7D305E03968514A531C3B60114242
:1091280068D07868C00702D07868A84378603E2085
:10913800A0642574257502A8FAF7DAFD002800D086
:10914800FEE70CCE474C2046083EFAF719FD0028EA
:10915800FED1B268F36820460830FAF711FD0028FE
:10916800FED13269736920461030FAF709FD0028EC
:10917800FED1B269F36920461830FAF701FD0028DC
:10918800FED1326A736A20462030FAF7F9FC0028CB
:10919800FED1B26AF36A20462830FAF7F1FC0028BB
:1091A800FED1326B736B20463030FAF7E9FC0028A9
:1091B800FED1B26BF36B20463830FAF7E1FC002899
:1091C800FED1326C736C20464030FAF7D9FC002887
:1091D800FED1B26CF36C20464830FAF7D1FC002877
:1091E800FED1326D736D50342046FAF7C9FC002861
:1091F8001DD0FEE7616A0818A9043A680A4290D0AF
:10920800626A82428DD23A680A428AD0626A82428F
:1092180087D23A680A4284D0626A824281D23A6826
:109228000A4200D17DE7626A8242E6D379E7E8071D
:109238007968014379607868FFF784FD03B0F0BD71
:10924800E4BD0008FC06002068000020E8090020B2
:109258008BC100081020024023016745AB89EFCD80
:08926800FAC3000000F0010848
:10927000F0B581B0544801F01BF80125290253488C
:10928000415A534E3184E021415AB184E221415A7E
:109290007184E421415A3185E621415AF18421212A
:1092A000C900415AF18583214900415A3186412143
:1092B0008900415A718581214900405AB085454F46
:1092C0007868002806D53846083843490160434984
:1092D000016078687D20C1004148426A52182B0421
:1092E0003C681C4215D0446A944218D23C681C4227
:1092F0000FD0446A944212D23C681C4209D0446A9E
:1093000094420CD23C681C4203D0446A9442E7D396
:1093100005E03A68334B5C1C3C601A4230D07968F7
:10932000C90702D07968A94379603F218164057437
:1093300005756846FAF7E0FC002804D02A4800F0DA
:10934000B7FF01B0F0BD326A736A284C2046FAF7C5
:109350001BFC00280FD1B26AF36A20460830FAF7E6
:1093600013FC002807D1326B736B10342046FAF7D8
:109370000BFC002820D01E4800F09AFF01B0F0BD81
:10938000426A5118AA043B681342C8D0436A8B4210
:10939000C5D23B681342C2D0436A8B42BFD23B68FE
:1093A0001342BCD0436A8B42B9D23B681342B6D059
:1093B000436A8B42E7D3B2E7E807796801437960F3
:1093C000786801B0F0BDC04668C40008FC06002003
:1093D000000000201020024023016745AB89EFCD3B
:1093E000E8090020FAC3000098C1000800F801084D
:0493F000FABD0008BA
:1093F400F0B58DB0024608466538444244410846FB
:109404006F3843424341234303D102206F2903D1E0
:1094140004E001206F2901D0652901D10A3000E060
:1094240009309A4D6A609A4E35600127BA023C03AE
:1094340065290492059406D06F2902D103214A02BA
:1094440001E000221446AC602A610021002B00D107
:109454007903E96000F080FC8E4B002202F090F862
:1094640000F032FC2A688C498A42069009DD8B4957
:109474008A420CD08A498A4209D08A498A4206D053
:1094840046E089498A4202D088498A4240D18424EC
:109494002859002846D1802000262E542868814966
:1094A400884233D1B8038449CA680243CA60CA688F
:1094B40002400892089808683843086008683840F1
:1094C40007900C970B960A960220039009900920A6
:1094D40040020890079805200007029008A901910E
:1094E400FAF7EAFC0C970B960A97039809900498EC
:1094F400089002980199FAF7DFFCFF2000066F49F3
:109504000A6882430A60F8066D490860604E09E003
:109514003A0249326648674900F0C8FE8424285953
:109524000028B8D02420285128680168B943016074
:10953400FBF75CF8012827D0A86A002801D0FBF7C4
:10954400D1FAB903286882680A438260F903826801
:109554008A43826001685B4A0A400260F9054268F6
:109564000A434260B90602680A430260FF242106E6
:1095740042690A4006990A4342610168394301601D
:10958400FBF7ACFB002801D072B6FEE731680A464F
:1095940080329068202809D18B680598834202D1D3
:1095A4000869002802D01078012803D14C4800F043
:1095B4007DFEFEE70D465C3500200690C8661770F8
:1095C4002C806C8027368E65002B0AD03E07B34270
:1095D4000BD03E03B3420DD10E69002E0DD13A4C8F
:1095E4000BE00E69002E07D107E00C69002C03D0B4
:1095F4003F2402E0A88001E07F24AC80D0602224D4
:1096040094600E68B4683C43B460380204907C07EC
:10961400486EA04202D1A889FF280DD9059883423B
:1096240002D1086900282DD02B4B069C049D147090
:109634000B672035334610E00598834202D1086950
:10964400002821D0224D069C3346083314700D6740
:1096540030680499084330603D070D4A26201454AD
:109664004720C0001F4911508D2080001B49115014
:109674001868284318609484D46114841C3294714B
:109684000DB0F0BD134BD0E7104DDCE7DC08002033
:10969400C004002000000C40FF4B0040004C004080
:1096A4000080004000380140004400400048004071
:1096B400F2C0000818C200083410024018E400E0A8
:1096C40000E100E0FFFF00FCFF010000A94F0008DB
:1096D4006D4E0008DFB4000875B40008700B00205C
:0896E4001CBE0008060A00206C
:1096EC00F0B58AB098480168CC6908680990486858
:1096FC00012007900007069088680890230753D034
:10970C000698401C089A104001252A02164620365D
:10971C00099F3E40064347D03A4056425641E20725
:10972C00079A00D03246002A05D10D628C22864F52
:10973C00BE582E43BE50089A15406A426A41A6078D
:10974C00079E00D51646002E08D102220A628C22F2
:10975C007D4EB658042737437B4EB7506A426A4158
:10976C006507079D04D4002D04D0002B0CD41BE0FE
:10977C001500FAD104220A628C22734FBD580226BE
:10978C002E43BE50002B0FD5421E9041099A9206D3
:10979C00079A00D40246012A06D1082008628C22BE
:1097AC00694DAB580343AB500125E80504902005E7
:1097BC0013D50898049A1040AA06099B1A40101851
:1097CC000BD0E8020862882020225F4B1A508420BC
:1097DC001A505E4805755E4A85540395202027462D
:1097EC00059007401ED00898069A1040099A059BD0
:1097FC001A40024316D04520C000544A13588825FD
:10980C00514E7559222D00D094E0FE2B00D991E0D9
:10981C00D3184D6A27269D554D4B039DD55413588F
:10982C005B1C1350802326461E402ED00898049AA9
:10983C001040099A1A40024327D0444800688422F9
:10984C008258212A14D1024656321588002D0FD089
:10985C0005680195056D02952D780092019A956227
:10986C00029A551C0565009A1088401E108007E06E
:10987C00006802689A43026002684025154305603F
:10988C00324D23200001039A2A5402934025099A51
:10989C002A4050425041620600D507900798002894
:1098AC000DD10868A84308608420274B059A1A50EC
:1098BC00284800220270882022241C505A678C22CF
:1098CC002148805800282AD0882422201E4B185169
:1098DC00002F09D0089B079106991940099F059BF9
:1098EC001F400F4307991CD1002E18D0089B049AD7
:1098FC001340099A029E32401A4310D00A68AA43B8
:10990C000A608421104B059A5A50185126200F4991
:10991C0000220A5423200001039C0C545A670AB0FD
:10992C00F0BD8869082303438B61002006498850E9
:10993C000AB0F0BD8869082202438A61802326465A
:10994C001E40A2D072E7C046DC080020C0040020F4
:08995C0031020000E6040020C6
:109964000122D20703004B403AD430B4431A01D247
:10997400C01AC9184B004400240EFF2C29D0002C17
:1099840024D01B0E20D0E31A182B1DDC090211432E
:10999400C40D000210435D4219350A00AA40D209E1
:1099A400D940451801D36D080234013CE405280A66
:1099B4000121C9072D062A438A4160414100090E4D
:1099C400FF2901D3C00DC00530BC7047C00FC007CC
:1099D400FAE74202F8D07F2000010C300005F3E7DB
:1099E400A4465140431A02D25340C01AC9184B002E
:1099F400090211431B0E4400240EFF2C41D0002BFE
:109A040010D05B421B19012B10D322D1C30D40028D
:109A1400401A10D3DB050100400AC90591415841A1
:109A2400644670472442FBD10020F9E7C30D40028D
:109A34004900401AF4D0002101314000FCD38C428B
:109A440004D95B1ADB05400AC018E9E7180AC00705
:109A5400E6E7192BE4D801330C00D940DC414C4033
:109A6400012C4941C30D00021043441A01D4A4003F
:109A74006408013BDB05200A2406944158416446EE
:109A84007047FF2B01D04102CAD07F2000010C3067
:049A94000005C5E71D
:109A98000122D2075140014B18470000699900087C
:109AA80030B405004D400124E407254042004B0036
:109AB800120E32D01B0E3CD0FF2A33D0FF2B3FD0E2
:109AC800D21800022043000A09022143090AC4B23D
:109AD8004C43000AC3B24B43000A4843210A5B18AF
:109AE800190A091801D44900013A080A7F3A2ADB01
:109AF800FE2A0FD2D2051C43240601D0012421439B
:109B0800C9B280295041802901D14008400028432A
:109B180030BC7047FF20C005F9E71B0EFF2B0AD0A9
:109B28002800F5E7400206D1FF2BF3D1490202D104
:109B3800F0E7FF2AF4D17F2000010C300005E7E7A9
:109B48004902F8D1E6E743020132E9D15B12023358
:089B5800E6D9D805E4E7C04698
:109B600030B405004D400124E407254042004B007D
:109B7000120E26D01B0E34D0FF2A2DD0FF2B35D04D
:109B8000D21A000220430902214343084908A00DCC
:109B90005B1A02D2013A5B005B185B008B4200D378
:109BA0005B1A4041F9D37F3222DDFF2A06D2D2056B
:109BB000C91A8B425041284330BC7047FF20C00572
:109BC000F9E71B0E03D0FF2B12D1490210D07F20E2
:109BD00000010C300005EFE74002F8D1FF2BEDD17A
:109BE000F5E7FF2AEAD14002F1D1E7E74902EED1D9
:049BF0002800E1E781
:109BF40002000A43520008D0884204D140000121E7
:109C04000906C84201D90020704701207047C046A8
:109C1400012212064300DA4211D84B00DA420ED870
:109C240002000A43520008D003D288428041013026
:109C34007047814280410130704701207047002005
:049C44007047C0465F
:109C4800012212064300DA420FD84B00DA420CD840
:109C580002000A43520008D003D2814280414042A8
:109C68007047884280414042704700207047C04694
:109C7800012212064300DA420FD84B00DA420CD810
:109C880002000A43520008D003D288428041404271
:109C98007047814280414042704700207047C0466B
:109CA80041000DD2090E7F390AD449421F3105D42B
:109CB80000020122D2071043C8407047C8177047F6
:049CC80000207047C1
:109CCC004A0010D2520D03231B02FF33D21A0AD4BE
:109CDC0052421F3209D4400DC90208430123DB074D
:109CEC001843D040704700207047D0177047C046CB
:109CFC00420017D2120E7F3A14D480231B06202A5E
:109D0C0006DA52421F3200021843D040002170473D
:109D1C0052423F3209DB010219430800D041D140C5
:109D2C0048407047002001007047D0170100704771
:109D3C009D2201000AD002D4013A4900FCD5D2057B
:109D4C00080A0906494100D3012950417047C04611
:109D5C0042221201033A010007D002D4013A001842
:0C9D6C00FCD51205C30A40059918704789
:109D7800BD22094210D003D4013A00184941FBD54D
:109D8800D2050128804101300143080A09064941EA
:109D980000D3012950417047004908473D9D0008FC
:109DA8004B1801225205DA4217D25B0D0722D20165
:109DB8009B1A0FD9FF2B13D2DB05CA0FD207134307
:109DC8000903020D1143490AC200524100D9013169
:109DD800C8187047C80FC007704706D1002804D1BB
:109DE800C80F0002FF30C00570470123DB070A00D7
:109DF800C900400F084398431A4010435B0A1843B0
:049E08007047C04699
:109E0C00F0B581B00A464149C30D5C1EFD2C58D8F3
:109E1C00FD24E443D50DFF3DA54252D306460E402A
:109E2C00491C0140964260D90091DCB20123DD054A
:109E3C00002C03D0691E0840284309E0AE4206D22C
:109E4C009F05641E7000BE420646FAD300E0304601
:109E5C00D10DCEB2002E03D0691E0A402A4308E071
:109E6C00AA4206D29F051146761E4A00B9421146F7
:109E7C00FAD3B4420ADD811A02D4904201D109E02E
:109E8C000146641E4800B442F5DC3446861A03D4FD
:109E9C00904202D1009A11E00646AE4206D29905D4
:109EAC00641E70008E420646FAD300E03046002C49
:109EBC001FDD611E009A8018C9054218104601B0BA
:109ECC00F0BD4500124CA5421BD25500AC42F5D951
:109EDC0006460E40FF24E5050E4CAE4213D0002E74
:109EEC000BD10A420246E9D10DE000D001460A46E8
:109EFC00E4E7191BC8400021DCE70A4003D0AA4262
:109F0C008ED10246DAE72246D8E7C046FFFFFF7F34
:089F1C00010000FF0000C07FFE
:109F2400C10DC9B24A1EFE2A19D27E2903D80028BF
:109F340013DA104870479529FCD87F390C4A0A4136
:109F44000240134603D5094B5B1CCB40D318884011
:109F5400400200D01A46104670470020704700297E
:109F6400E8D10121C90708407047C046FFFF7F00C0
:089F7400000080FF000080BF27
:109F7C0030B5514343435C18010C130C0D005D4389
:109F8C00641992B2514380B242430D0C0904521829
:109F9C0065415843010C00048018694130BDC0462E
:109FAC00CA1751408B1A17D0C1174A4094464840E3
:109FBC00411A48081A0000E052008242FCD90020E5
:109FCC0000E05208914200D3891A40419A42F8D1DC
:109FDC0062465040801A704710B500F07DF810BDF5
:109FEC0007B5FFF7DDFF0EBC4243891A00BDC04622
:109FFC000A0015D00300400800E052008242FCD950
:10A00C00002000E052089B1A06D340418A42F9D145
:10A01C00704752089B18F8D200188A42F9D1704741
:08A02C0010B500F059F810BD59
:10A0340038B504004D42FFF7DFFF4543611938BDD1
:10A04400002B09D1002907D110B51100FFF7F0FF4B
:10A054000A000021002310BD70B400240125ED077F
:10A06400002B07D1002905D0834203D2130000221C
:10A074002C0000250026A419994200D1904212D93F
:10A0840092185B4103D2EE076D086408F3E7DE071C
:10A094005B08520892190126F6079B1903E0DE07B4
:10A0A4005B0852089219801A994103D364416D41A7
:10A0B400F5D30FE024196D410AD2DE075B0852087C
:10A0C400921980185941F5D364416D41E7D301E0F9
:10A0D4008018594102000B002000290070BC704711
:08A0E400002000217047C04676
:10A0EC0003490868002800D0704702480860704790
:08A0FC00400B0020480B00207E
:10A104007F2805D8034A125C0348405C104070471E
:0CA1140000207047E8C40008BAC2000830
:10A120007F2805D8034A125C0348405C1040704702
:0CA1300000207047E8C40008BAC2000814
:10A13C00411C02780130002AFBD1401A7047C046FE
:10A14C00002A03D0013A8B5C8354FBD17047C04684
:10A15C0000220B0011001A00002A02D0013A81548F
:04A16C00FCD170476B
:10A17000F0B581B00022002933D00378002B30D015
:10A18000032302469A4316680024E5438707FF0E1F
:10A19000BD40ED43354306461E4071180429009327
:10A1A0000AD3124EAF19104BAB433B4204D1091FE7
:10A1B0005568121D0329F5D82B060DD02B041B0E54
:10A1C00007D02B021B0E06D02B0E009C04D00424BB
:10A1D00002E0012400E002248C4200D30C46101A55
:10A1E0000219104601B0F0BD80808080FFFEFEFEA7
:10A1F000F0B581B004467F20C605002C00960FD034
:10A20000E11722464A40571AC6050A4DF80704D0FE
:10A2100029683046FFF748FC06462D1D7F08F5D11A
:10A2200000983146FFF79CFC002C00D4304601B06A
:08A23000F0BDC04678B3000840
:10A23800F0B503AF93B06E46F51D2135F41D3934E2
:10A2480074613362F261F160306100F0FDFEB0606C
:10A25800C21D07218A436946B1616946881A706040
:10A268008546F41D1D34002124222046FFF776FF81
:10A278000B487169F2680A6048600A4828603069CA
:10A288002862B06868617068E8602046F169326ADF
:10A2980000F01EF8B1698D46FC1F053CA546F0BDCF
:08A2A80057B90008FFFFFF7F1A
:10A2B00083B010B581B0044603A80EC005480068FD
:10A2C00003AA0092214601F073FA01B010BC02BC4F
:08A2D00003B00847640B0020F5
:10A2D800F0B59FB014460F4600211590016001208B
:10A2E80002020C92460282020392C20202920322E6
:10A2F8000A9292020592020317924203079282037E
:10A3080004920090C00316900891C84301900F96DC
:10A318003978252908D0002901D100F060FE7F1C7A
:10A32800159801F0E4F9F3E7FF1C089BB81E0578BF
:10A338002A46203A102A2BD880219200184602A3D8
:10A348009A5803469746C04695A30008B5A3000847
:10A35800B5A30008AFA30008B5A30008B5A300087B
:10A36800B5A30008A1A30008B5A30008B5A3000879
:10A37800DFA30008A5A30008B5A30008A9A3000847
:10A38800B5A30008B5A30008ADA3000840210AE062
:10A398005E2D179907D009E0169904E0202102E004
:10A3A800102100E031460B437F1CBFE77F1E294682
:10A3B8003039C9B20929139419D800240A216143F4
:10A3C8006C18303C791C3D782A46303AD2B20A2AB9
:10A3D8000F46F3D30CE001CC0028139401D51021CB
:10A3E8000B43C1174840441A781E057800E0002442
:10A3F80000202E2D08D13D782A2D07D17D78BF1C4D
:10A40800139901C9139113E00E9018E07F1C294697
:10A418003039C9B209290FD80A21414368183038A0
:10A42800791C3D782A46303AD2B20A2A0F46F3D32D
:10A4380000280E9001D502E00E900C9803431846B0
:10A44800E1172A46683AD301D2B252089A18D2B212
:10A45800092A2BD8920002A39A5803469746C04669
:10A4680091A400089BA40008A5A40008C5A400089E
:10A47800C5A40008C5A400089FA40008C5A4000836
:10A48800C5A400089FA400083D78682D10D10820B5
:10A4980008E0022003433D787F1C0FE03D786C2DD7
:10A4A80009D1022003437D78BF1C07E0034605E07D
:10A4B8007F1C042201E07F1C012213438C43462D9C
:10A4C8000B941BDD2946633915292BD8139CC046EC
:10A4D8007944097949008F44460B421CC30A0B0A88
:10A4E8000A0A0A5966730A0A810A830A0A2E0FE7BA
:10A4F800049803430021099119467AE0442D1598E0
:10A50800139C08DD452D28D0462D00D000E707987C
:10A518000343029824E0252D00D080E2252101F094
:10A52800E6F8F5E6472D139C00D197E0582D00D0AA
:10A53800EEE607980343CE4A782D00D1203219065B
:10A54800C81709900C98034201D0CA48034019461D
:10A558000498099B134009934BE007980343039819
:10A568000343059A7EE0264624780B98421E159DE3
:10A57800284619461292149301F00BF928462146F1
:10A5880034460F9E01F0B3F8241DDFE0180700D50C
:10A5980049E29807159801682068016000D446E2EE
:10A5A8000021416043E20C980342194601D0B148AA
:10A5B80001401A06D217302010400990049818E07C
:10A5C800069718060C990B43C017232101400991DF
:10A5D80004CC1394002708200E90B2E101CC8DE042
:10A5E8000C98034201D0A34803401946049800225E
:10A5F800099202220A400142069706D1002A09D18F
:10A60800231D002722461C460AE0002A12D104CC4A
:10A61800D01715E0E21D07239A43576814460834FB
:10A6280013684A0714D408220A4000D0DBB2002A73
:10A638000FD1FCE0E41D07229443226860680834C7
:10A648004B0708D40B0700D5DDE013460746DDE0CD
:10A658009BB20027EBE013B21204D6E0079803433D
:10A66800059A13430C98034201D00E9800E0062087
:10A6780014931340991A4A424A410E92002800D076
:10A688000E90E41D0720844303CC083CFFF788FBA9
:10A698002546044601F024F808351395002820467D
:10A6A8000ED00021FFF7E4FA149B1A4607990A40D6
:10A6B800002813D0002A704800D070482C461BE0B0
:10A6C80001F005F8002846D00798149B03426C480F
:10A6D80000D06C486C490B402C460FE0002A6B49AF
:10A6E80000D06B49002A01D0694800E067482C4631
:10A6F800401C9A0600D5084663490B400028654E61
:10A7080000D0064619465B48014014910C98034254
:10A718001394304602D1FFF70DFD02E00E99FFF7C2
:10A7280023FD05460B98441B15981499224601F001
:10A7380030F8002D129407D0159C3178204600F08F
:10A74800D6FF761C6D1EF8D1139C0F9E1498C00678
:10A7580000D4DDE55DE10126204601F080F80546DC
:10A76800002801D0F007444012961EA9204601F0A7
:10A7780094F81E980A9948430A21FFF713FC0646E5
:10A788001E90002D03D060201499014314910025D8
:10A7980020462946FFF72AFA002818D1701CFFF72F
:10A7A80023FD01462046FFF74BFA00281E9806D0E5
:10A7B800411C1E91801CF2E71E98401E1E90FFF758
:10A7C80013FD01462046FFF753FA0028F4D1149AE6
:10A7D80016460598064012998B029E4200D128E140
:10A7E800864209D11E980E99814200DC22E104219B
:10A7F800C943884200DC1DE112930398024200D04D
:10A8080020E10E9D06E253B21206D717002F05D499
:10A818008A060AD44A060AD5202007E000225B42AD
:10A82800BA412D200990174601E02B2009901A46BD
:10A838000C98014201D00F4801400B460C98014288
:10A84800139401D00E9800E0012000246E2D0E9084
:10A8580039DD6F3D092D00D994E0C0467D442D793E
:10A868006D00AF44196E8F8F8F8F368F8F6EC046F5
:10A8780058300000FFFDFFFFCCC20008C7C2000827
:10A888008CC5000888C50008FFFEFFFFD6C2000877
:10A89800D1C20008E7BA00081046384372D0D00881
:10A8A80079074018014607201040303018AA105583
:10A8B800C808FF087A0780180A463A43641C002A29
:10A8C8000A46EFD15EE0582D3BD0642D01D0692DAA
:10A8D80058D11046384355D01946169801400D9165
:10A8E8000021149314463B460D9800280F4608D0C3
:10A8F80008460A990840032803D118A82C21C155F5
:10A908007F1C0A2200252046194612932B46FFF782
:10A9180095FB1094044611910A222B46FFF72AFB57
:10A92800109A101A3021014318A8C155791C092022
:10A93800801A12988541119F0F9E149BD3D30C4601
:10A9480020E0104638431CD007981D460342FA48B9
:10A9580000D0FA48134611093A07891800240A4614
:10A968000F211940415C18AB195511093F093B07E4
:10A97800C91813463B43641C002B1346EFD12B46E2
:10A9880000E00024099A511E104688410B99091BC2
:10A99800FF2A00D9491E069F081A0E990D1BE917B0
:10A9A8008D43421B3342149305D11598194600F084
:10A9B800F0FE149B0022099E310A129204D01598C9
:10A9C80000F095FE129A149B002E3146159E04D075
:10A9D800304600F08CFE129A149B3046194600F05F
:10A9E800D8FE302130462A4600F0A3FF012C0ADBAE
:10A9F800641C18A80019801E0178304600F077FE04
:10AA0800641E012CF5D81498C006139C0F9E00D420
:10AA18007EE420211598129A00F08BFF78E4002D2F
:10AA280000D075E4EBE22068159909680170241DCF
:10AA38006EE41E98119626282ED12046CC49FFF7A1
:10AA48008BF82FE01E980E2800DDE3E0C0430E9936
:10AA58000E18102E00DB1026100600D5D9E0002EA7
:10AA6800354600D1D6E03046FFF7BEFB2146FFF75A
:10AA780017F83F210906FEF771FFFFF74FFABD49A6
:10AA8800FFF7C0F900252946FFF7B0F8002800D1E4
:10AA9800BFE0761EE7D1BDE04042FFF7A5FB2146A7
:10AAA800FEF7FEFF064600252946FFF79FF8002817
:10AAB800139C15D1304600F013FE0028304611D003
:10AAC8000021FFF7D5F8149B1A4607990A40002879
:10AAD80000D196E0002AA84800D10DE6A7480BE669
:10AAE800099527E00995A34C2146FFF78FF81E9D8D
:10AAF80000280BD030462146FFF72EF8064621469F
:10AB0800FFF784F86D1C0028F4D11E957F20C4053A
:10AB180030462146FFF7ACF800280BD0304695495F
:10AB2800FEF7BEFF06462146FFF7A2F86D1E002875
:10AB3800F4D11E950598119981420E9801D00546C9
:10AB480000E0451E8B4C0028294600D100211191B8
:10AB58004842FFF749FB019900F083FE3146FEF7B2
:10AB6800FDFE06462146FFF751F8002807D01E983B
:10AB7800401C1E9030462146FEF7EEFF0646149A0A
:10AB880011980D96002839D0119502990B468033FB
:10AB980013408B4200D0ABE0102800DB10200546A4
:10ABA800FFF722FB3146FEF77BFFFFF7A3F8109073
:10ABB80008430998119000D19AE00A2200231098BE
:10ABC8000E46FFF73BFA002D00D190E01A4300D063
:10ABD8008DE0119531460A2200231098FFF72EFACE
:10ABE80010900C460A220023FFF728FA1198401EFD
:10ABF80011907DD01A432146EDD079E00998119043
:10AC080076E0002A5E4900D05E49002A6DD05D4892
:10AC18006EE535461E9810386942884200DC0846C1
:10AC2800FFF7E2FA019900F01CFE2146FEF796FEB6
:10AC380004461E98401CFFF7D7FA01462046FEF747
:10AC4800FFFF1E99002800D0491C1498002911956F
:10AC580011D4112914D3084610381E901020401A18
:10AC6800FFF7C2FA2146FEF71BFFFFF743F8064637
:10AC78000C46002012E00D9400261E9634460FE084
:10AC880000201E902046FFF735F8254606460C465C
:10AC9800FFF76EF801462846FEF7FAFE0D90149865
:10ACA80012998843DB49083100250A4608326D1C91
:10ACB8000B684968F31A23468B411146F6D2109562
:10ACC800119B002B0099149A01D1D1B2C9095206DF
:10ACD800920F01D1494200E0C9431E9A891A0B9A82
:10ACE800D21A5118491B024676E0C74800E511956B
:10ACF800119D002D0098149A01D1D0B2C0090B996A
:10AD0800491B081A411F1E9C17980242129E01D126
:10AD180010963FE00E91032120461091FFF762F94B
:10AD2800881C042822D8C04678440079400087440B
:10AD380007132B071300C04678C5000868C500082C
:10AD4800641E1E940D98B149FEF7AAFE0D900E9947
:10AD5800491E022010901AE0A41E1E940D98AC49BA
:10AD6800FEF79EFE0D900E99891E10E000200CE063
:10AD78009976967E00002041CCC20008C7C2000820
:10AD8800D6C20008D1C20008012010900E99149A6A
:10AD9800E81785435006800F119500D0491E0E9183
:10ADA800F502204600F08BFD632802DD0E98401E58
:10ADB8000E9014980D9CA84314902046FEF79AFF15
:10ADC800254606460C46FEF7D3FF01462846FEF701
:10ADD8005FFE149A0D900E99C8170D4685430F987B
:10ADE80010300242149208D1012906DB202115985F
:10ADF80000F07DFC6D1EF9D1149A40201040910698
:10AE080003D400280AD0202104E0002801D02D21F5
:10AE180000E02B21159800F06AFC149AD0060AD499
:10AE2800002D08D03021159800F061FC6D1EF9D175
:10AE380000200E9000E00E951099491E0D46C8009E
:10AE4800744A111849681258B01A2046884101D22C
:10AE5800302007E03020B61A8C41401CB31A234634
:10AE68008B41F8D2C1B2159800F041FC2946002D5B
:10AE78001498E2D10146029801401291159E0BD018
:10AE88001E98012808DB401E1E903021304600F035
:10AE98002EFC1E980028F6DC802014990840119C8E
:10AEA80020430E9D4BD02E21304600F020FC102C64
:10AEB800264600DB1026F0173446844312980028F3
:10AEC80001D1204601E01E98201AFFF78DF90146AE
:10AED80011981094001B0B90012E23DB0D98FEF7A0
:10AEE800DFFDFEF707FF04460E46109B5B1ED800E9
:10AEF800484A111849681258A01A304688411293D6
:10AF080001D2302007E03020A41A8E41401CA31A39
:10AF180033468B41F8D2C1B2159800F0E8FB129B7A
:10AF2800002BE3D10B980028159E119807D0109993
:10AF38000C1A3021304600F0DAFB641CF9D3039870
:10AF4800149901423BD00798014201D0452100E005
:10AF58006521159C204600F0CAFB1E980028204653
:10AF680004D42B2100F0C3FB1E9805E02D2100F02E
:10AF7800BEFB1E9840421E9064280FDB6421FFF739
:10AF880039F801463031159E304600F0B0FB1E9866
:10AF98006421FFF727F808461E9100E026460A219B
:10AFA800FFF700F801463031304600F0A0FB1E984C
:10AFB8000A21FFF717F83031304600F098FB002DD2
:10AFC800139C0F9E01D1FFF7A3F9159C2021204661
:10AFD80000F08DFB6D1EF9D1139CFFF799F9159CB4
:10AFE800E068002805D006CC083C914201D2089AB6
:10AFF8004254204600F0C0FB20681FB0F0BD00F0AE
:10B00800BBFB0198F9E7C046D6C200080000204102
:08B018000000C842C03000082E
:10B02000084B1B6883420AD0074B1B68834206D03B
:10B03000064B1B68181A431E984140427047002077
:10B04000FCE7C046680B0020640B00206C0B00205E
:04B0500040207047E5
:0CB0540010B5006800F0C8F810BDC04640
:10B0600003230F480F4A036143610F4B8261C361A1
:10B070008023DB000362002383624362C3620266B3
:10B080000A4A426610228266094A0367C36643671A
:10B090001178013AC1540133102BF9D17047C046E1
:10B0A00034080020A8B30008C0000020240B0020B2
:04B0B000D7B300080A
:10B0B400F8B54746CE46C56883680400406899469B
:10B0C4005B1B80B50E00170098464019934207D9C0
:10B0D400FFF73AF8ED19E560C0BCB946B046F8BDD3
:10B0E4001A00FFF731F84B463100ED19ED1A2A002A
:0CB0F40060684144FFF728F8EDE7C04613
:10B10000F8B54746CE46002380B5884607001600AE
:10B110009946C56884681BE0013B5B1B641BB44215
:10B1200000D934009C4200D91C00786822004146B6
:10B130004019FFF70BF82D19A144A044361BBC6839
:10B14000631B5A1E93415B421D40FD60002E06D0DA
:10B150003B699D42E0D3013B1B195B1BDEE7484680
:08B16000C0BCB946B046F8BDC1
:10B1680070B50600431C5C00E4181D4BE400E018B1
:10B178007400A419E4001B19DC6A1500012C06D020
:10B18800022C1FD0002C10D00024200070BD9A6A19
:10B198005C6AA2421FD9013A121B2C00954200D9C1
:10B1A80014002200FFF782FFEFE79A6A5E6AB24254
:10B1B8000CD9013A961BB542E7D82A00FFF776FF6B
:10B1C8002C00E2E7FFF798FF0400DEE71B6AD218BD
:10B1D800013A961BEFE71B6AD218013A121BDCE70B
:04B1E8003408002007
:10B1EC00F8B50B4B04001B780D001600002B0CD08F
:10B1FC00EFF31087012181F3108832002900200021
:10B20C00FFF7ACFF87F31088F8BDFFF723FFEFE7DC
:04B21C0034080020D2
:10B22000072904D9024B416018600023036070476E
:04B23000440B0020AB
:10B23400000000000000000000000000000000000A
:10B2440000000000000000000000000000000000FA
:10B2540001000000020000000300000004000000E0
:10B2640006000000070000000800000009000000BC
:10B2740000000000000000000000000000000000CA
:10B2840001000000020000000300000004000000B0
:10B29400000000000400000002000000080000009C
:10B2A400004B0000650001000100740EF00A420E1C
:10B2B400100E540B800CC409280AF401C201320098
:10B2C40046006AFF9CFF5802100EFA0000000000BE
:10B2D400000000000000000000000000000000006A
:10B2E400DB090020DC090020DD090020DE09002044
:0CB2F4002ABE000820B3000800B30008C8
:10B3000005A100080BB9000817B9000821A1000821
:10B3100023B900082FB90008FBB80008CFB800080F
:10B320002CBE0008A7C20008A7C20008A7C20008D8
:10B33000A7C20008A7C20008A7C20008A7C2000849
:10B34000A7C20008A7C20008FFFFFFFFFFFFFFFF23
:10B35000FFFFFFFFFFFF00002EBE000859C20008DC
:10B360007ABA000876C20008D1BA0008A8C200085C
:08B37000B1C20008D8BA0008C0
:10B37800000020410000C84200401C4620BCBE4CD2
:08B38800CA1B0E5AAEC59D74EC
:10B3900003480449091A08B5FFF742FF0CBC1847D7
:08B3A000100C00201010002029
:09B3A8005465726D696E616C0060
:10B3B100455845433A20466163746F72792052655E
:07B3C10073746F72650A004E
:10B3C800000000000000545452205245474745539E
:01B3D8000074
:0FB3D900455845433A20524553544152540A00B7
:02B3E800FEE77E
:02B3EA00FEE77C
:02B3EC00FEE77A
:02B3EE00FEE778
:02B3F000FEE776
:02B3F200FEE774
:02B3F400FEE772
:02B3F600FEE770
:02B3F800FEE76E
:02B3FA00FEE76C
:02B3FC00FEE76A
:02B3FE00FEE768
:02B40000FEE765
:02B40200FEE763
:02B40400FEE761
:02B40600FEE75F
:02B40800FEE75D
:02B40A00FEE75B
:02B40C00FEE759
:02B40E00FEE757
:02B41000FEE755
:02B41200FEE753
:02B41400FEE751
:02B41600FEE74F
:02B41800FEE74D
:02B41A00FEE74B
:02B41C00FEE749
:02B41E00FEE747
:02B42000704773
:10B4220030B584214158212918D102465632938AD7
:10B43200002B13D0016802E05B1E1C040ED014889E
:10B44200002C0CD0CC692406F6D5046D25788D62CB
:10B45200641C04651488641E1480EDE730BD01206D
:10B46200C0058A6882438A600868402202430A60F3
:02B4720030BDEB
:10B4740010B5882141582229016810D102465E3254
:10B484005388496A1940836D19701188491E1180C7
:10B49400816D491C81651188002905D010BD88691A
:10B4A400082202438A6110BD0246883209214B01F9
:10B4B40001680C689C430C608B680124A3438B6077
:10B4C4002023136000220267C36E012B03D10B6893
:0AB4D4001024A3430B60C26610BDF4
:10B4DE0010B588214158222901680FD102465E32EB
:10B4EE0053884C6A1C40836D1C801488641E148023
:10B4FE009B1C83651288002A05D010BD886908221E
:10B50E0002438A6110BD0246883209235B010C6832
:10B51E009C430C608B680124A3438B602023136033
:10B52E0000220267C36E012B03D10B681024A343C4
:06B53E000B60C26610BDA7
:02B54400FEE720
:02B54600FEE71E
:02B5480070474A
:02B54A00704748
:10B54C0008D1002806D1F54204D801D3002A01D134
:10B55C006D0D09D10020C143090DC904F0BDF9D10D
:10B56C001242F7D1640DF5D00020C14349054908BA
:10B57C00A6E000206146F0BDF0B50127FF070E00E4
:10B58C005E403E40B446BE0A4C18DD18F442D7D299
:10B59C00F542E4D2640DECD06D0DEAD06419C90209
:10B5AC003943460DC0023143DB023B43DB0A10B486
:10B5BC008E4685B297B26F43140C6C433E0CA419A3
:10B5CC00260C2404BFB227439CB26C43A419190C5B
:10B5DC006943250CA4B249190D04090C6419000C1B
:10B5EC0095B245433E0C76193743BFB2360C150C59
:10B5FC004543AD19A6B2240CAD192E0437432E0CBD
:10B60C0036199DB24543AD19ACB22E0C89191D0CDF
:10B61C0045436D182E04290C3443704680B295B204
:10B62C0045433E0C76193743BFB2360C150C4543D7
:10B63C00AD19A6B2AD19240C2E0437432E0C3619B5
:10B64C009DB24543AD19ACB22E0C89191D0C454366
:10B65C006D182E043443290C75462D0C90B268439A
:10B66C003E0C80190604BFB23E43070CA0B23F1833
:10B67C00120C6A43D019020C80B2240CA4189AB292
:10B68C006A43121914042043120C89181B0C6B43C7
:10B69C00C91810BC01273D05294203D1B6194041F8
:10B6AC004941013CFF077D0D013D641B0BDB6D0027
:10B6BC00AC4209DA240500254208BE4168416141CB
:0AB6CC0066463143F0BD54E74EE737
:10B6D600FF2109064000884201D80020704701205A
:02B6E6007047AB
:0EB6E8000121090640004118484248417047C0
:10B6F60030B581B0044668460170206900280FD035
:10B706000CCC083C9A4233D26269531C6361815463
:10B71600A069616981422BD1204600F02EF827E00E
:10B72600E068002809D00CCC083C9A4220D2551C6F
:10B736009D4200D1002181541AE0A068002808D05B
:10B746000CCC083C9A4213D2551C9D420DD0C9B26E
:10B756000CE0236A002B0BD003CC083C884207D2AE
:10B76600694601222046984702E000219200815056
:0AB776002068401C206001B030BDC7
:10B7800010B54269002A07D00446036A002B01D095
:0AB79000216998470020606110BD98
:10B79A0080B5CB0606D4890501D5302100E02021E9
:06B7AA0000F0C6F880BDAE
:10B7B00070B514460D460646FEF798FC0146304625
:0AB7C0002A462346FEF738FD70BD4F
:08B7CA00F7F7D3FCF7F7C7FC09
:10B7D200806A816D40220A438265C16D04220A4358
:04B7E200C265704785
:10B7E60010B58421415821290DD1014656310A88C8
:10B7F600002A09D00268036D1C7894625A1C0265FF
:10B806000888401E088010BD0068016880229143A8
:0CB816000160016840220A43026010BD7E
:08B8220080B5FDF762FF80BD57
:08B82A0080B5FDF75EFF80BD53
:10B83200F0B581B01E4615460C4607461846FFF77E
:10B84200EEFB0146002000290AD46543A54207D336
:10B85200304639462A46FFF7FCFB2146FEF7CDFB70
:04B8620001B0F0BD84
:04B86600C00F704758
:10B86A0010B5FD22D343C20DD2B21446FF3C9C420E
:10B87A0008D351184A1EFD2A05D8FF22D205904343
:10B88A00C905084310BD0122D20710400129F9DB7E
:08B89A00FF21C905401810BD93
:10B8A200C20DD2B2FF2A01D0002A02D100220A60C0
:10B8B20070477E3A0A60FF21C90588433F21090685
:04B8C2004018704773
:08B8C600C1174840401A704709
:10B8CE0010B5002A0DD00446097848B200280AD4D3
:10B8DE00002C00D02160002119605960411E884162
:0CB8EE0010BD002010BD0120C04310BDA3
:10B8FA00024601207F2901D9C04370471170704761
:0CB90A00014661391A2900D2203870472C
:0CB91600014641391A2900D22030704748
:0CB92200014661391A2900D22038704714
:0CB92E00014641391A2900D22030704730
:10B93A0070B5012A09DB0C460546561C28462146E5
:0CB94A00FFF7D4FE761E012EF8D870BD69
:10B9560010B50C46436A01212046FFF767FF10BD6C
:10B96600010002000400060008000A000C00100096
:08B976002000400080000001E8
:10B97E006E6F7420616C6C6F7765642C20706172D1
:0FB98E00616D746572206C6F636B6564210A00D4
:10B99D0048414C5F434F4D50315F53746172742079
:07B9AD004552524F520A00FF
:10B9B40048414C5F434F4D50325F53746172742061
:07B9C4004552524F520A00E8
:10B9CB00434F4E564552544552204552524F523AD0
:10B9DB0020434F4E5645525445525F535441525497
:0BB9EB005550204552524F52210A00D7
:10B9F600434F4E564552544552204552524F523AA5
:10BA060020434F4E5645525445525F4552524F526F
:10BA16005F4F55545055545F564F4C545F544F4FDB
:07BA26005F484947480A0090
:10BA2D0042617474657269652063686172676564EB
:10BA3D0021204379636C65636F756E7465722B2B72
:03BA4D00210A00CB
:10BA500048414C5F4144435F53746172745F444D8D
:07BA6000413A204F4B0A00A0
:10BA67002D3E4D65737361676520746F2073686F32
:03BA7700727400E6
:10BA7A004A616E75617279004665627275617279A2
:10BA8A00004D6172636800417072696C004D6179A2
:10BA9A00004A756E65004A756C7900417567757361
:10BAAA00740053657074656D626572004F63746FDC
:10BABA00626572004E6F76656D62657200446563F9
:07BACA00656D62657200006A
:07BAD100414D00504D000043
:0FBAD80025612025622025652025542025590051
:07BAE700286E756C6C29004C
:10BAEE00443A5C70726F6A656B74655C6563735F14
:10BAFE00677265656E506F7765725061636B5C65DA
:10BB0E0063735F63656C6C4D6F6E5C6669726D77A7
:10BB1E006172655C447269766572735C53544D3321
:10BB2E0032473078785F48414C5F4472697665726F
:10BB3E005C5372635C73746D3332673078785F6810
:0ABB4E00616C5F636F6D702E630081
:10BB5800443A5C70726F6A656B74655C6563735FA9
:10BB6800677265656E506F7765725061636B5C656F
:10BB780063735F63656C6C4D6F6E5C6669726D773D
:10BB88006172655C447269766572735C53544D33B7
:10BB980032473078785F48414C5F44726976657205
:10BBA8005C5372635C73746D3332673078785F68A6
:0EBBB800616C5F666C6173685F65782E630078
:10BBC600443A5C70726F6A656B74655C6563735F3B
:10BBD600677265656E506F7765725061636B5C6501
:10BBE60063735F63656C6C4D6F6E5C6669726D77CF
:10BBF6006172655C447269766572735C53544D3349
:10BC060032473078785F48414C5F44726976657296
:10BC16005C5372635C73746D3332673078785F6837
:0ABC2600616C5F6770696F2E6300A8
:10BC3000443A5C70726F6A656B74655C6563735FD0
:10BC4000677265656E506F7765725061636B5C6596
:10BC500063735F63656C6C4D6F6E5C6669726D7764
:10BC60006172655C447269766572735C53544D33DE
:10BC700032473078785F48414C5F4472697665722C
:10BC80005C5372635C73746D3332673078785F68CD
:0ABC9000616C5F756172742E630031
:10BC9A00666163746F726520726573746F72652072
:0ABCAA002850696E292E2E2E0A0084
:10BCB4004558453A2053746F726520706172616D06
:06BCC400657465720A00C0
:10BCCA00455845433A204170706C79204D422050C6
:0ABCDA006172616D657465720A0005
:10BCE400455845433A20526573657420436F756E19
:06BCF400746572730A0082
:10BCFA0048414C5F4441435F5374617274204F4B17
:02BD0A000A002D
:10BD0C0042414C414E4345525F496E6974204F4B42
:02BD1C000A001B
:10BD1E00434F4E564552544552204552524F523A79
:10BD2E0020434F4E5645525445525F4552524F5244
:10BD3E005F4F55545055545F564F4C545F544F4FB0
:06BD4E005F4C4F570A0094
:10BD540042617474657269652064697363686172B1
:06BD6400676564210A007E
:10BD6A004D696E75746520496E74657276616C6C86
:0ABD7A0020636865636B73210A0003
:10BD84004E6577204D696E20566F6C74616765202F
:0ABD940025642053617665640A00FF
:10BD9E004E6577204D617820566F6C746167652013
:0ABDAE0025642053617665640A00E5
:10BDB8004669727374207374617274206465746563
:06BDC800637465640A00CB
:10BDCE00454550524F4D2046554C4C2052455354EC
:06BDDE004F5245210A004E
:10BDE400454550524F4D2053544F524520434F4EDA
:06BDF400464947210A0048
:10BDFA004572726F72207768696C65207361766923
:10BE0A006E67206461746120746F20666C61736868
:02BE1A000A001C
:0EBE1C0075617274206572726F72200A0D00DB
:02BE2A004300D3
:02BE2C002E00E6
:10BE2E0053756E646179004D6F6E6461790054755F
:10BE3E006573646179005765646E6573646179003A
:10BE4E005468757273646179004672696461790031
:0ABE5E00536174757264617900008D
:10BE6800443A5C70726F6A656B74655C6563735F96
:10BE7800677265656E506F7765725061636B5C655C
:10BE880063735F63656C6C4D6F6E5C6669726D772A
:10BE98006172655C447269766572735C53544D33A4
:10BEA80032473078785F48414C5F447269766572F2
:10BEB8005C5372635C73746D3332673078785F6893
:09BEC800616C5F6164632E63008C
:10BED100443A5C70726F6A656B74655C6563735F2D
:10BEE100677265656E506F7765725061636B5C65F3
:10BEF10063735F63656C6C4D6F6E5C6669726D77C1
:10BF01006172655C447269766572735C53544D333A
:10BF110032473078785F48414C5F44726976657288
:10BF21005C5372635C73746D3332673078785F6829
:09BF3100616C5F6461632E630022
:10BF3A00443A5C70726F6A656B74655C6563735FC3
:10BF4A00677265656E506F7765725061636B5C6589
:10BF5A0063735F63656C6C4D6F6E5C6669726D7757
:10BF6A006172655C447269766572735C53544D33D1
:10BF7A0032473078785F48414C5F4472697665721F
:10BF8A005C5372635C73746D3332673078785F68C0
:09BF9A00616C5F646D612E6300AF
:10BFA300443A5C70726F6A656B74655C6563735F5A
:10BFB300677265656E506F7765725061636B5C6520
:10BFC30063735F63656C6C4D6F6E5C6669726D77EE
:10BFD3006172655C447269766572735C53544D3368
:10BFE30032473078785F48414C5F447269766572B6
:10BFF3005C5372635C73746D3332673078785F6857
:09C00300616C5F74696D2E63002D
:10C00C00443A5C70726F6A656B74655C6563735FF0
:10C01C00677265656E506F7765725061636B5C65B6
:10C02C0063735F63656C6C4D6F6E5C6669726D7784
:10C03C006172655C447269766572735C53544D33FE
:10C04C0032473078785F48414C5F4472697665724C
:10C05C005C5372635C73746D3332673078785F68ED
:0DC06C00616C5F756172745F65782E630012
:10C0790066756C6C20726573746F72652E2E2E0A4C
:01C0890000B6
:10C08A00455845433A2053746F726520776974683E
:05C09A0020736E0A0096
:10C09F00455845433A2053617665206C6F636B209A
:05C0AF006B65790A0039
:10C0B400455845433A2044656C6179206F662031C8
:10C0C400207365636F6E642120446576696365201F
:0DC0D4006D7573742072657365742E0A001B
:10C0E100554E4B4E4F574E20434F4D4D414E440AF6
:01C0F100004E
:10C0F20057726F6E6720706172616D6574657273DD
:10C102002076616C75653A2066696C65202573201E
:0DC112006F6E206C696E652025640D0A00BB
:10C11F0048414C5F4441435F53657456616C75658C
:05C12F00204F4B0A0047
:10C1340048414C5F4441435F5374617274204552DB
:05C14400524F520A00F9
:10C1490044432044432057616E646C6572206E6FCE
:10C15900742072756E6E696E672C207374617274C7
:09C1690020696D70756C730A0009
:10C1720070726576696F757320636F6E666967208A
:09C1820070726573656E740A00A9
:0DC18B0057726974696E6720534E210A00D7
:10C198004572726F72207768696C652064656C659A
:10C1A80074696E67206C6F672064617461206172C6
:0DC1B800656120696E20666C6173680A0085
:10C1C50048414C5F41444345785F43616C69627205
:10C1D5006174696F6E5F53746172743A204F4B0AD4
:01C1E5000059
:10C1E6004572726F722048414C5F4144435F5374FD
:09C1F6006172745F444D410A00BE
:10C1FF002D3E4D657373616765207769746820778D
:09C20F00726F6E67206372630018
:10C21800443A5C70726F6A656B74655C6563735FE2
:10C22800677265656E506F7765725061636B5C65A8
:10C2380063735F63656C6C4D6F6E5C6669726D7776
:10C248006172655C7372635C6D6F646275732E6393
:01C2580000E5
:10C2590053756E004D6F6E00547565005765640027
:0DC26900546875004672690053617400004E
:10C276004A616E00466562004D617200417072004F
:10C286004D6179004A756E004A756C00417567000C
:10C29600536570004F6374004E6F7600446563000B
:01C2A6000097
:01C2A7000096
:09C2A800256D2F25642F25790076
:09C2B10025483A254D3A255300B9
:0DC2BA000007032004170201085710408000
:05C2C7002D494E460068
:05C2CC002D696E660003
:05C2D1002B494E460060
:05C2D6002B696E6600FB
:01C2DB00FF63
:04C2DC0085310008A0
:10C2E000443A5C70726F6A656B74655C6563735F1A
:10C2F000677265656E506F7765725061636B5C65E0
:10C3000063735F63656C6C4D6F6E5C6669726D77AD
:10C310006172655C447269766572735C53544D3327
:10C3200032473078785F48414C5F44726976657275
:10C330005C5372635C73746D3332673078785F6816
:0CC34000616C5F6164635F65782E6300D0
:10C34C00443A5C70726F6A656B74655C6563735FAD
:10C35C00677265656E506F7765725061636B5C6573
:10C36C0063735F63656C6C4D6F6E5C6669726D7741
:10C37C006172655C447269766572735C53544D33BB
:10C38C0032473078785F48414C5F44726976657209
:10C39C005C5372635C73746D3332673078785F68AA
:0CC3AC00616C5F74696D5F65782E630042
:08C3B80001010103070100006F
:08C3C000080402040801010158
:10C3C8007265616420636F6E6669672E2E2E0A009F
:10C3D800455845433A205265736574204D696E206F
:10C3E800616E64204D61782056616C7565730A0032
:10C3F80048414C5F434F4D50315F53746172742014
:04C408004F4B0A008C
:10C40C0048414C5F434F4D50325F537461727420FE
:04C41C004F4B0A0078
:10C420004E6577204D696E2054656D702E20256411
:08C430002053617665640A00E7
:10C438004E6577204D61782054656D702E202564F7
:08C448002053617665640A00CF
:10C45000486F757220496E74657276616C6C2063EA
:08C460006865636B73210A009B
:10C46800454550524F4D2053544F5245204C4F474D
:08C478002044415441210A0057
:10C4800048414C5F41444345785F43616C69627247
:10C490006174696F6E5F53746172743A20455252D1
:04C4A0004F520A00ED
:10C4A4004572726F722C2072656164206F6E6C79B4
:0CC4B400205265676973746572210A00EC
:10C4C00050726F7465637465642052656769737434
:10C4D00065722C207772697465206E6F7420616CB0
:08C4E0006C6F776564210A000E
:10C4E80020202020202020202068282828282020DC
:10C4F8002020202020202020202020202020202034
:10C5080048101010101010101010101010101010EB
:10C51800848484848484848484841010101010108B
:10C5280010818181818181010101010101010101E4
:10C538000101010101010101010101101010101098
:10C5480010828282828282020202020202020202B5
:10C55800020202020202020202020210101010205D
:10C568003031323334353637383941424344454621
:10C578003031323334353637383961626364656651
:04C588004E414E00D2
:04C58C006E616E006E
:10C5900000B506480649884205D00268043003B455
:10C5A000904703BCF7E708BC18470000DCC200084E
:04C5B000E0C20008DD
:10C5B4001DC6000800000020480B00002FC600081C
:10C5C400480B0020D8C5000891B3000891C50008A5
:04C5D4006B310008BF
:10C5D80018F4B20008F4B20008F4B20008F4B2008B
:10C5E80008F4B200080024F4000AFE000F340B001F
:10C5F80020380B00203C0B002000000202FD00FD4B
:10C6080002010101FB00E702040100000102980099
:04C61800800000009E
:10C61C00206861680834002200E042540139FCD5DE
:02C62C00704755
:10C62E002068616808340A780131802A11D009D354
:10C63E000B7801315242FF32013203700130013A60
:10C64E00FBD5F0E70B78037001300131013AF9D5D3
:04C65E00E9E7704751
:10C66200FFFFFFFFFFFFFFFFFFFFFFFFFFFFFFFFD8
:10C67200FFFFFFFFFFFFFFFFFFFFFFFFFFFFFFFFC8
:10C68200FFFFFFFFFFFFFFFFFFFFFFFFFFFFFFFFB8
:10C69200FFFFFFFFFFFFFFFFFFFFFFFFFFFFFFFFA8
:020000040801F1
:04EFFC00CF5D82B4AF
:040000050800B7CB6D
:00000001FF
